:040FF8000060020093
:040FFC0000E007000A
:020000022000DC
:106000000000012079630200616302006363020003
:10601000656302006763020069630200000000001C
:10602000000000000000000000000000818F02005E
:106030006D630200000000006F63020071630200E4
:1060400073630200736302007363020073630200F0
:1060500073630200736302007363020073630200E0
:1060600073630200736302007363020073630200D0
:1060700073630200736302007363020073630200C0
:1060800035B10200736302007363020073630200A0
:106090007363020073630200C1DF020073630200D6
:1060A0007363020073630200736302007363020090
:1060B0007363020073630200000000000000000030
:1060C0007363020073630200736302007363020070
:1060D000B1AA0200736302007363020000000000B3
:1060E00000000000000000000000000000000000B0
:1060F00000000000000000000000000000000000A0
:10610000000000000000000000000000000000008F
:10611000000000000000000000000000000000007F
:10612000000000000000000000000000000000006F
:10613000000000000000000000000000000000005F
:10614000000000000000000000000000000000004F
:10615000000000000000000000000000000000003F
:10616000000000000000000000000000000000002F
:10617000000000000000000000000000000000001F
:10618000000000000000000000000000000000000F
:1061900000000000000000000000000000000000FF
:1061A00000000000000000000000000000000000EF
:1061B00000000000000000000000000000000000DF
:1061C00000000000000000000000000000000000CF
:1061D00000000000000000000000000000000000BF
:1061E00000000000000000000000000000000000AF
:1061F000000000000000000000000000000000009F
:10620000364937480A1A02D0072291438D4635494C
:1062100035480A1A06D00722914381F309880222E1
:1062200082F3148831483249324A00F045F8324846
:106230003249334A00F040F832483349334A00F0DB
:106240003BF833483349344A00F036F83348344990
:10625000344A00F031F834483449354A00F02CF81B
:1062600034483549354A00F027F835483549002289
:1062700000F02DF834483549002200F028F8344861
:106280003449091A082903DB002202600430016046
:10629000314A90471F482049884205D0026804309F
:1062A00003B4904703BCF7E700208646EC46002085
:1062B00000212A4A9047FEE7884207D0521A05D0AB
:1062C000037801300B700131013AF9D170478842EF
:1062D00002D002700130FAE7704700000000012090
:1062E00000F800200000012000000120901B0300A6
:1062F000CC57002020580020D8630200D863020049
:1063000036E50200901B0300CC570020CC5700203C
:1063100038E6020038E6020038E6020038E60200FD
:1063200038E6020038E6020038E6020038E60200ED
:10633000901B0300E41B030020580020205800207D
:10634000205800202CA000202CA000202CA00020F1
:106350002CA000202CA00020A1630200E1920200EA
:10636000FEE7FEE7FEE7FEE7FEE7FEE7FEE7FEE705
:10637000FEE7FEE7704700BF1048804710484FF027
:106380000701884385460F4880470F48016841F45C
:1063900070010160BFF34F8FBFF36F8FFFF730BF06
:1063A0000A480B490B4A884207D0521A05D0037895
:1063B00001300B700131013AF9D170477563020069
:1063C000000001206DB2020088ED00E024E602002A
:0863D000B8570020CC57002053
:1063D8007047000007B5044B0093044A402300F0BF
:1063E80032F803B05DF804FBF9630200215800207D
:1063F8002DE9F84389461446B2B10F4B0F4E0325D9
:10640800002743F00108224609EB0701002004F0A9
:1064180003F80744241A48B933782BB14FF47A406B
:10642800C047013D02D13570BDE8F88301233370C0
:10643800002CE8D1F8E700BF40E602002058002011
:10644800704704F01DB8F0B595B01C4616460846CE
:106458000D4601F06CFD1A9B0D93CDE908640024EC
:106468002346082205A928460A948DF82C400C9446
:1064780001F086FD079B0293BDF81830ADF80C308B
:10648800BDF81A30ADF80E309DF814308DF8114073
:1064980003F00302012A1DD1BDF81440059EC3F381
:1064A800C203C4F383148DF81030A20008230EA988
:1064B800284601F065FDC6F3952608AB00932246F1
:1064C80002AB0EA9304600F027FC284601F033FD48
:1064D80015B0F0BD022AF8D1BDF81640C3F3C203C7
:1064E800A4098DF810300827082C264628BF08264E
:1064F8003B4632460EA9284601F042FDA41B08ABD4
:1065080002AA31460EA8374400F06AFC002CEBD1F1
:10651800DBE7000008B5FFF794FF0421064800F008
:1065280065FB002803DA0549412000F0EBFD044B28
:1065380001225A7108BD00BFE4E5020054E60200DA
:10654800CC570020037813F0040216D003F003039D
:10655800012B03D0022B09D0012070470A6800885C
:106568000232C0F3831002440A60F5E70B684288E0
:10657800023303EB92130B60EEE7104670470000FE
:106588002DE9F04F89B00646871C08A80023484C1F
:1065980000F8113D0D46009200F046FD23682B607F
:1065A800D4E90123DFF810811344226801339B1AD0
:1065B800A8F1040BA8F10809BB421AD3009A0023DA
:1065C800002A6DD0012262F3010343F0040366F34D
:1065D80089132168A2689DF80F000A4003320F440E
:1065E80044F82230276000F04FFD012009B0BDE8D3
:1065F800F08F0121404600F072FE584600F088FEF8
:106608000DF1200A484600F083FE60684AF8100D34
:10661800A5682840033004EB80005146FFF792FF3D
:1066280002460498002AF4D105EA000304EB830328
:10663800811CDB6805930130054004EB850503F0F8
:106648000303012B0491ED6823D0022B08D01949CC
:1066580001924FF4BF7000F055FD019A154607E00E
:10666800BDF816309B0903332D0C01EB93030493FB
:10667800484600F050FE08B1049B63602946404636
:1066880000F02DFED4E901231344226801339B1A3C
:1066980092E7BDF81430C3F383132D0C0B44E6E7DF
:1066A800022262F3010343F0040366F39F5390E769
:1066B80034590020C3E60200506900200D4B0E48F3
:1066C80040F2FF3241F2180110B59A6000225A5088
:1066D80041F21401C3E900225A5003F581531A709C
:1066E80001F0DEFB044610B9044801F05FFC2046C7
:1066F80010BD00BF34590020BCE502001CE70200B1
:1067080030B50A4C71B10A4A0A49121BD208002353
:106718009A4201D1002030BD31F82350854202D081
:106728000133F5E7034654F83300F4E74CE502007B
:10673800BCE50200B8570020094B013903EBC00043
:10674800032909D8DFE801F00A020406042070478B
:1067580000797047407970470020704702207047E1
:106768004CE50200034BD3E90030C31A58425841A4
:10677800704700BF345900202DE9F04387B0FFF778
:10678800F1FF0646002840F00681844D41F21803C7
:10679800E850BFF34F8F6868AC68DFF8188206AF1F
:1067A80047F8100D2040033005EB80003946FFF70D
:1067B800C9FE029B18B1D8F80020002A61D004EA6B
:1067C8000302991C013305EB8202234005EB830386
:1067D800D268DB68049302F00303022B0392029150
:1067E80067D1BDF80E306E484FEA9318B8F1500FD4
:1067F800C14628BF4FF0500969F38F1309F108010A
:10680800ADF80E3001F064FB0746002800F0AD80BB
:1068180001F08DFB03A900230822384601F09AFBFA
:10682800029924EA01060136B600B1453AD95FFA61
:1068380089F9A6B3F6B2A9EB0609214003315FFA3C
:1068480089F4B146574E05EB810108234A4638467C
:1068580001F080FB36B109F108032246314638467B
:1068680001F078FB029B08F1030803EB98030293FD
:1068780041F21803EB58002B4FD141F21003EC58AA
:106888005EE02A689A4204D86A60304607B0BDE8DC
:10689800F08304EA0300033005EB800086E74149F2
:1068A8003446D2E72140033108234A4605EB8101EB
:1068B800D5E7012B59D1BDF80C303948C3F3831102
:1068C800062928BF062161F3891302318900ADF832
:1068D8000C3001F0FDFA0746002846D001F027FBEE
:1068E8000023082203A9384601F034FB0026BDF82E
:1068F8000C20C2F38312B31C96424FEA8303B7D22B
:1069080002994A1C21400331029205EB81010422BD
:10691800384601F01FFB0136E9E7384601F00BFB6A
:10692800FFF720FF80F00100C6B2AEE7E3685B79AD
:1069380023B1236839461B6820469847E3681C68DA
:10694800002CF3D1384601F0F6FA06A800F8114DEC
:1069580000F06AFB41F21803EB580BB9029B6B601D
:106968009DF8070000F090FBDAE741F21003EC58BD
:1069780054B90D4B0D480E49C01AC008000440F028
:10698800020000F087F8CBE7236820469B68984709
:10699800E3681C68ECE7002677E700BF345900205D
:1069A800BCE50200405900204CE502004CE502001D
:1069B80028E702004C6900202DE9F74F2F4D80464B
:1069C8000F46914601A9012218469B46D5F808A012
:1069D800FFF7D6FD00283DD0019C0026A11C5E458E
:1069E80006EB010240D10021254800F042FC80F36B
:1069F800100B244B244A4FEA18499B1AB9EBD30FC2
:106A080004D3224940F2A31000F07CFB631C03EA84
:106A18000A0305EB830349EA0B42DA6004EA0A0336
:106A28000333012115F8232068F3C50205F8232054
:106A380035F8232066F3891225F8232055F82320FA
:106A480067F39F2245F8232061F301026FF3820266
:106A580005F823200E4B1B781BB1FFF78DFE00288D
:106A6800FBD103B0BDE8F08F0AEA020205EB82020F
:106A780059F82630D3600136B1E700BF34590020F9
:106A880050690020BCE502004CE50200C3E60200A4
:106A98005469002000231A46FFF78EBF13B502ACD5
:106AA800012344F8042D2246FFF786FF02B010BDEB
:106AB80007B5CDE9002302236A46FFF77DFF03B03F
:106AC8005DF804FB1FB5CDE90123069B039301AADA
:106AD8000323FFF771FF05B05DF804FB1FB5CDE98F
:106AE8000023069B0293079B03936A460423FFF740
:106AF80063FF05B05DF804FB7FB5CDE90123089B72
:106B08000393099B04930A9B059301AA0523FFF7A6
:106B180053FF07B05DF804FB2DE9F3478046304C7E
:106B2800D01C8A46174601A900228008A568FFF7ED
:106B380027FD002840D0DDF80490A66809F102007E
:106B4800019001362840361AB6000330B74204EBEC
:106B580080003BD83A46514607F03BFC00212148CB
:106B680000F087FB80F3100009F101032B4004EBD0
:106B780083034FEA184242EA0040D86005EA090355
:106B8800033304EB830214F8231068F3C50104F8F7
:106B9800231034F823106FF38F1124F82310518831
:106BA80067F38F11518014F82320022161F3010249
:106BB8006FF3820204F823200B4B1B781BB1FFF7FD
:106BC800DBFD0028FBD102B0BDE8F0873246514614
:106BD80007F0FFFBBA1B0AEB060104F10C00BBE748
:106BE80034590020506900205469002030B541F222
:106BF80010030F49CA580023144644B9C4682371C6
:106C08005AB941F2100548512260184630BDE4686F
:106C180025799D4206D02468EFE7D2681168216083
:106C28001060F2E701330A2BE6D14FF0FF33ECE7AF
:106C38003459002038B541F21002094B9C5803F52D
:106C48008152012313701D4604B938BDE3685D7194
:106C5800236820465B689847E3681C68F4E700BF30
:106C680034590020037A052B10B50C460FD0437A0F
:106C780023B1084A0849204600F0F8FB0749204696
:106C880000F0F4FB2046BDE8104000F0DDBB002A10
:106C9800F8D0F3E773E70200BA0F030095E70200A4
:106CA800C38873B504460D4633B1144A009214499B
:106CB800144A284600F0DAFB217A05291CD0637AA9
:106CC8004BB1A088FFF738FD0F4B104953F820202F
:106CD800284600F0CBFB227A0D4BA08853F822609F
:106CE8000021FFF70DFD0B4903463246284602B046
:106CF800BDE8704000F0BABB02B070BD73E7020097
:106D080080E7020078E7020040E70200BA0F0300BC
:106D1800A4E7020098E702002DE9F04385B01F467A
:106D28000C9D002306460C46904695F80C902B7354
:106D380029463846FFF7B4FFB8F1060F09D8DFE84F
:106D480008F00412181F283340003146284600F086
:106D58008DFB002229463846FFF784FF85F80C9002
:106D680005B0BDE8F08322683146284600F07EFB76
:106D7800EFE7D4E900233146284600F077FBE8E73F
:106D8800A36800933146D4E90023284600F06EFB3F
:106D9800DFE7E3680193A36800933146D4E9002351
:106DA800284600F063FBD4E723690293E368019364
:106DB800A36800933146D4E90023284600F056FB27
:106DC800C7E76369039323690293E3680193A368A0
:106DD80000933146D4E90023284600F047FBB8E782
:106DE80008292DE9F84F80460E4617461C463AD822
:106DF800002593F80C901D7319461046FFF750FFB5
:106E0800DFF884A0DFF884B0AE422ED918F8052048
:106E18005946204600F02AFB0135082DF4D11849BF
:106E2800DFF86CB0204600F021FB4FF0000A564511
:106E380020D918F80A507E2D03D8284607F08EFA74
:106E480000B92E252A465946204600F00FFB0AF1C4
:106E5800010ABAF1080FEAD1012221463846FFF7A4
:106E680001FF84F80C90BDE8F88F5146204600F0E9
:106E7800FDFAD1E70349204600F0F8FAE7E700BF3A
:106E88006EE702006CE702006AE7020064E70200AE
:106E980070E7020012F0030310B511D1094C22600B
:106EA8004C1CE400A4B22244074C2260074A137029
:106EB800074A1370074A1080074A1846118010BD08
:106EC8000720FCE7F8690020F4690020F069002039
:106ED800006A0020FC690020FE6900202DE9F347C4
:106EE8002B4D2B888B4206460C4617464BD302A8DF
:106EF8004FF0000800F8018D00F096F8254B264A5F
:106F080018781178CBB2254909888B4238BF0133EC
:106F1800C0B238BF5FFA83F840452ED092F800809F
:106F28001378DBB2994286BF0133DBB200231370BA
:106F38009DF8070000F0A8F84FF6FF73984524D095
:106F4800DFF860A0DAF800304FEAC80903EB09025D
:106F580043F83870A6B19CB1114B28881B682246AB
:106F680008FB0030314607F034FADAF800304B44B9
:106F780000209C8002B0BDE8F0874FF6FF78D7E785
:106F880000209080F6E70920F4E70420F2E700BF2C
:106F9800FC690020006A0020F0690020FE690020DA
:106FA800F4690020F8690020F8B5124C124D264605
:106FB80022782B789A4200D1F8BD23780F48104ADE
:106FC800078812680F48DBB219B202EBC10C0068DF
:106FD80052F83120BCF8041003FB070090470A4A16
:106FE80023781288DBB29A4286BF0133DBB20023D2
:106FF8003370DDE7006A0020F0690020FC6900209A
:10700800F8690020F4690020FE690020EFF3058389
:10701800C3F308032BB9EFF31480C04300F0010059
:10702800704701207047000070B50446FFF7EEFF77
:10703800012803D01049432000F064F8EFF31086CC
:1070480072B60E4A9068012398B993600C4B0D4DA7
:10705800D3F8801029401160C3F88050D3F8841009
:1070680051604FF0FF32C3F88420207006B962B631
:1070780070BD2370FAE700BF09E80200046A002027
:1070880000E100E0FC06FFBD10B50446FFF7BEFFB7
:10709800012803D00949512000F034F8084B9A68B8
:1070A8005AB154B9EFF3108172B6064A18681060E5
:1070B800586850609C6001B962B610BD09E80200CA
:1070C800046A002000E100E030B53AB11368DB4300
:1070D8000B4C0144884204D1D84330BD4FF0FF33F4
:1070E800F6E710F8012B5340082213F0010F14BFE4
:1070F80025460025013A85EA5303F6D1EAE700BFA1
:107108002083B8ED07B5ADF8000001916A4600216B
:1071180044F2020002F0B6F803B05DF804FB10B5C3
:1071280061B1B2FBF3F403FB1424A4B244B9C0E97F
:10713800001484608281C381204610BD0E20FCE7C4
:107148000920FAE782B050E8022FC188B2EB324F2B
:107158004FF0000317BF92B241EA014142EA0141F0
:1071680004E04268B2EB324F08BF012340E8021244
:10717800002AE8D18DF807309DF80730002B0CBFA6
:107188001120002002B0704737B550E8013F9DB28A
:10719800C48925448489A54228BF2D1B0489A5429A
:1071A80002BFBFF32F8F002207E0C5EA030540E8BE
:1071B8000154002CE9D14FF001028DF8032001930E
:1071C800019B9DF803200B6002F0FF0322B10B889E
:1071D8000068184403B030BD1846FBE70A884B889E
:1071E8009A4209D150E8012FC2EA024240E801233D
:1071F800002BF7D1012070470020704737B550E8C1
:10720800023F1FFAA3F5C488A54202BFBFF32F8F20
:1072180000220DE0C48925448489A54228BF2D1B7E
:10722800C3EA054540E80254002CE8D14FF00102BA
:107238008DF803200193019B9DF803200B6002F059
:10724800FF0322B14B880068184403B030BD1846CC
:10725800FBE70A884B889A4209D150E8022FC2EA14
:10726800224240E80223002BF7D10120704700207A
:10727800704750E8002F0B4640E8003C9CF0000F98
:10728800F7D11046704750E8002F42EA010340E862
:10729800003C9CF0000FF6D11046704750E8003FC4
:1072A80043EA010240E8002C9CF0000FF6D110469A
:1072B800704750E8002F02EA010340E8003C9CF0C8
:1072C800000FF6D11046704750E8003F03EA01026C
:1072D80040E8002C9CF0000FF6D11046704750E8AB
:1072E800003F03EB010240E8002C9CF0000FF6D1B0
:1072F8001046704750E8003FA3EB010240E8002C1D
:107308009CF0000FF6D1104670470121FFF7BBBF74
:107318000121FFF7C3BF0021FFF7CBBF0021FFF713
:10732800D3BF000010B50446002834D003681BB949
:107338001A49FF20FFF7E6FE636823B917494FF49F
:107348008070FFF7DFFEA36823B9144940F20110EB
:10735800FFF7D8FEE36823B910494FF48170FFF7AF
:10736800D1FE238A23B90D4940F20310FFF7CAFE64
:10737800D4E9012321689B1ADBB20A60013BDBB226
:10738800FF2B226802D10020107110BD1168481C23
:1073980010600B70F2E70E20F7E700BF67E8020005
:1073A80037B5054620B913494FF49270FFF7AAFE86
:1073B80002A8002400F8014DFFF736FE2A686B6822
:1073C800116899420ED9481E106011F8014CEB68FB
:1073D800298A01FB0434AB6811791B1ADBB2994284
:1073E80038BF13719DF80700FFF74EFE204603B023
:1073F80030BD00BF67E8020037B50C46054620B926
:10740800104940F24710FFF77DFE24B90D494FF4AB
:10741800A470FFF777FE02A8002300F8013DFFF7EC
:1074280003FE2A681368591C1160EA68A41A2A8A9C
:10743800B4FBF2F41C709DF80700FFF725FE03B0BB
:1074480030BD00BF67E8020010B5044618B9064908
:107458003120FFF757FEA2682AB1636921682069C5
:1074680098470023A36010BDB7E802000EB433B5F7
:10747800059D044618B912494220FFF743FE636987
:107488001BB90F494320FFF73DFE23681BB90C4980
:107498004420FFF737FE63681BB909494520FFF709
:1074A80031FE3DB102AA06AB42F8043D294620460A
:1074B80000F076F802B0BDE8304003B0704700BF76
:1074C800B7E802000A2938B504460D4602D10D2155
:1074D800FFF7F8FFA3682268591CA160D554D4E9C6
:1074E80001329A4204D32046BDE83840FFF7ACBFCA
:1074F80038BD00002DE9F84F9946DDE90A431746E3
:10750800824688460A460126BA420FD24E4538BFFF
:107518004E4613F0010B01D164B900240125B9F1DD
:10752800010F1AD909F1FF397D43F8E7B2FBF7F2E9
:107538000136E9E79B070ED5B9F1000F0CBF3025DE
:107548002025A642EAD2013C29465046FFF7BAFF59
:10755800002CF6D1E1E72025F3E7B8FBF5F39F42CD
:10756800E2D9DFF83890B8FBF5F3504619F8031064
:1075780005FB1388FFF7A6FFB5FBF7F5002DF2D141
:10758800BBF1000F02D00CB1A64201D3BDE8F88FC1
:1075980020215046013CFFF795FFF4E7FDE8020083
:1075A8002DE9F74F0E469046054620B9AC494FF4F1
:1075B800A270FFF7A7FD6B6923B9A9494FF4A3701F
:1075C800FFF7A0FD2B6823B9A54940F24710FFF744
:1075D80099FD6B6823B9A2494FF4A470FFF792FD97
:1075E800002E00F03A8116F8011B002958D02529F1
:1075F80040F0D180002702E047F0010716463246E6
:1076080012F8013B2D2BF7D0302B04D02B2B05D1B2
:1076180047F00407F2E747F00207EFE700242A2BB8
:1076280006F101021BD1D8F80030191D1B68C8F8F3
:1076380000101C44164633782E2B1CD101364FF00F
:10764800000A314611F8012BA2F13000092814D89C
:107658000A2303FB0A23A3F1300A0E46F1E712F8C6
:10766800013CA3F130010929E5D80A2101FB0434C2
:10767800303C1646D3E74FF0000A324612F8011B99
:1076880001F0FB0068281646F8D0692916D054D8AE
:10769800582970D00ED825297DD03378002BA2D157
:1076A8002B7B002B00F0D980284603B0BDE8F04FB3
:1076B800FFF7CABE632968D06429EED1D8F8002044
:1076C800D2F80090111D89EAE972C8F80010A2EBFF
:1076D800E9724FF0010B092A61DCD34538BFD34664
:1076E8002CB1B9F1000F01DB790700D5013CBA07CD
:1076F80002D5BAF1000F04D0FB0702D4002C54D1F4
:107708000024B9F1000F58DAC9F100092D212846E3
:10771800FFF7D8FE07F00302022A05D1BAF1000FDD
:1077280002D1002C4DD10024CDE9004753460A224E
:1077380049462846FFF7DEFEAFE7732954D016D82E
:107748007029AAD1D8F800301A1DC8F800203021B5
:1077580028461C68FFF7B6FE78212846FFF7B2FED8
:1077680000220823CDE9003221461022E1E77529DD
:107778002FD0782991D1D8F800100A1DC8F8002018
:10778800CDE90047534610222CE0D8F800301A1DE6
:107798001978C8F800202846FFF794FE7DE70A23E9
:1077A8000BF1010B92FBF3F295E7A345A9D2202137
:1077B8002846013CFFF786FEA0E77807AAD52B21CB
:1077C800A5E7A345B0D230212846013CFFF77AFE51
:1077D800A7E7D8F80010CDE900470A1DC8F800202F
:1077E80053460A220968A4E7D8F800301A1DC8F8D9
:1077F8000020F907D3F8009012D54F46A7EB090BE4
:1078080017F8011B41B9A345BFF447AF202128460B
:10781800013CFFF757FEF6E72846FFF753FEEDE772
:10782800B9F1000F17D0484606F051FE0746BC4292
:1078380000D954B909F1FF3919F8011F00293FF49B
:107848002CAF2846FFF73EFEF6E720212846013CEC
:10785800FFF738FEEBE74F46E9E703B0BDE8F08FE6
:107868000DE9020070B50D461646044618B90849D8
:107878005520FFF747FC1DB905495620FFF742FC84
:1078880025602B6831462046BDE87040184700BF88
:107898005AE902002DE9F041DDF818800E46174636
:1078A8001D46044618B922498820FFF72BFC1FB94A
:1078B8001F498920FFF726FC23681BB91C498A2029
:1078C800FFF720FC1DB91A498B20FFF71BFC6368E2
:1078D8005A68B5FBF2F302FB13531BB114498E200F
:1078E800FFF710FCB20703D011499120FFF70AFCFB
:1078F800BB0703D00E499220FFF704FCE3689E42C1
:1079080004D36B1E22693344934203D90849932058
:10791800FFF7F8FB2368CDF81880D3F80CE03A4657
:107928002B4631462046F446BDE8F041604700BF8B
:107938005AE902002DE9F0410D4616461F46044655
:1079480018B919499E20FFF7DDFB23681BB91649B2
:107958009F20FFF7D7FB1EB91349A020FFF7D2FBE2
:1079680063681B68013B2B4203D00F49A320FFF734
:10797800C9FBE3689D4207D363681B686A1E03FB63
:1079880006232269934203D90749A820FFF7BAFBC7
:107998002368D3F810E032463B4629462046F44691
:1079A800BDE8F041604700BF5AE902002DE9F04107
:1079B80008B10368C3B90E4E0E4B14229B1B00245A
:1079C800B3FBF2F3374602FB03F5A54201D10020D1
:1079D80008E03B5930190BB91434F6E7DB699847CE
:1079E8000028F9D0BDE8F081DB69BDE8F04118470F
:1079F800B8570020CC570020014B43600020704747
:107A0800BCE902000846704700207047024B18681E
:107A1800003018BF01207047106A002008B50248DE
:107A2800FFF77CFC002008BD106A002008B510464E
:107A38001A4606F0CEFC002008BD00002DE9F041F2
:107A4800804686B013480E4615461F46FFF75DFC74
:107A5800044630B1112018E006EB043000F092FC27
:107A68000134A542F8D10B48FFF758FCD8F8083084
:107A780000246BB1022268468DF80020CDE901464A
:107A8800CDE9034505979847204606B0BDE8F08143
:107A98001846FAE7106A00202DE9F041804686B0C2
:107AA80012480F4616461D46FFF72FFC0446D8B964
:107AB800AA083146384600F07DFC0C48FFF72EFC3A
:107AC800D8F8083073B101228DF800200C9A05927D
:107AD8006846CDE90147CDE903659847204606B0D9
:107AE800BDE8F0811846FAE71120F8E7106A00208F
:107AF80029DF704728DF704770B503689D6886B036
:107B080004460E466DB114220021684606F08AFC30
:107B1800A3680593237901962BB1012B0DD06846F4
:107B2800A84706B070BD01238DF800302369029381
:107B3800E368039363690493F1E702238DF8003047
:107B4800E3681B030293F5E7084670470020704777
:107B5800024B187A003018BF01207047006C0020D3
:107B6800034B187A0122B0FA80F05A744009704722
:107B7800006C002008B510461A4606F02AFC0020C2
:107B880008BD000008B514220021044806F04AFC8C
:107B98000348FFF7D7FA002008BD00BF006C00209B
:107BA800F06B002010B5094C094B43602046FFF7E5
:107BB800ACFB48B906F0E6F91C2320744FF4EE72CA
:107BC80004490548FFF7ABFA002010BD006C0020FF
:107BD800E8E90200146A0020F06B002070B5234D1C
:107BE800234E2B7A2C463BB922492348FFF706FB44
:107BF800306008B9686070BD0223237233681A794F
:107C080072B1012A22D018460321FFF775FF00231D
:107C18002372636017491848BDE87040FFF719BB25
:107C2800D3E90520121A142A28BF1422D3E9031510
:107C38009208012A014438BF01222844FFF758FF5F
:107C480050B11128DFD101232372D4E7D3E903020D
:107C58001044FFF74FFFF3E7237C002BCBD10146FD
:107C6800BDE87040022000F009B800BF006C002099
:107C7800186C0020146C0020F06B002038B5831EAF
:107C8800012B43D8224C237A002B3FD0022B09D159
:107C980003282ED01F4B1B680022E2601A793AB1E4
:107CA800012A20D0637C6BBBBDE83840FFF796BF44
:107CB800D3E905128D1A142D94BF521914329A6102
:107CC8009142EFD102284FF0000308BF19462372F2
:107CD800104B18BF0D211868FFF70EFF0E490F480B
:107CE800FFF7B7FADEE71A6901321A615B699A424F
:107CF800E7E7E3680133082B01D8E360D2E7002304
:107D0800E360DFE7BDE8384006F02CB938BD00BFB6
:107D1800006C0020186C0020146C0020F06B002010
:107D280000F0FD03012B08D1044B00225A74421EB7
:107D3800504250411874FFF751BF7047006C002043
:107D480010B5064C201DFFF7E0FA28B9637C1BB973
:107D5800BDE81040FFF742BF10BD00BF006C002017
:107D68002DE9F34180460D460F4801A916461F46E6
:107D7800FFF70AFA0446A8B11C22002106F052FBBC
:107D88002D0B0123237101A9C4F80080A760E560C9
:107D980066610548FFF722FAFFF7D2FF002002B01C
:107DA800BDE8F0810420FAE7F06B00202DE9F743E5
:107DB80081468846104801A917461E46FFF7E4F990
:107DC8000446B0B11C22002106F02CFB00250A9BBA
:107DD800A36001A92571C4F80090C4E9037866611D
:107DE8000548FFF7FBF9FFF7ABFF284603B0BDE8EE
:107DF800F0830420FAE700BFF06B00202DE9F74F6D
:107E080099469DF83030019388461746054618B9BB
:107E18002249B620FFF776F9EA8895F805B00BFBFA
:107E280002FBABF1040BCB4503D81C49C420FFF778
:107E380069F93E68B5F806A006EB09025A4509F14A
:107E4800040188BFABEB0906B1FBFAF43E600AFBFC
:107E5800141144B9AAEB0107B74228BF37462EB917
:107E680003B0BDE8F08F2D68013CF2E7019A0431B8
:107E780008EB0403681872B101463A461846F61B27
:107E880006F0A7FAB2453C442D6857464FF000016A
:107E980028BF3746E3E73A461946F0E714EA0200F6
:107EA800FFF740BAF8B546790146721E0546002329
:107EB80093422D6803D30024A64202D8F8BD0133AB
:107EC800F6E70F682846FFF797FA01343946F3E7D3
:107ED8002DE9F843068ACD1C0746FFF761FA043EF0
:107EE80035440446B5FBF6F5F0B14FF48073EDB2B6
:107EF8008380C680013D076081464FF00008A84591
:107F080012D23846FFF74CFA064648B16379013376
:107F1800637108F10108C9F8000007608146EEE7BF
:107F28002046FFF7BFFF34462046BDE8F88301210D
:107F38000430FFF7D4B910B5012104460430FFF727
:107F4800D9F910F0FF0F04D12046BDE81040FFF723
:107F5800A9BF10BD30B585B0144604AA002542F863
:107F6800044D0095FFF74AFF039BA34203D0034942
:107F7800F620FFF7C7F805B030BD00BF14EA0200CD
:107F880030B585B0144604AA012542F8044D009581
:107F9800FFF734FF039BA34204D003494FF48070DA
:107FA800FFF7B0F805B030BD14EA0200836800227C
:107FB8005A609A60C3E90422DA601A6070470000C8
:107FC80038B50D46044618B909495020FFF79AF804
:107FD8001DB907495120FFF795F82B686A68636057
:107FE800934208BF0023256008BF636038BD00BF07
:107FF80064EA020010B5044618B90B496320FFF77C
:1080080081F823681BB908496420FFF77BF8636887
:1080180043B12268916852680B449342636004BF7D
:108028000023636010BD00BF64EA02000D4930B54B
:10803800A1F594720225914201D800200EE08B1A16
:10804800DB1093FBF5F302EBC30452F833308342A1
:1080580005D802D204F10802EDE7606830BD214678
:10806800E9E700BF08EC020008B5FFF7DFFF024BA5
:10807800002808BF184608BDCDEA02002DE9F04FD8
:108088000022C9B04B780C781B0443EA0463CC780F
:1080980023438C7843EA042308AC0431A350043208
:1080A800402AEFD1234638AD996B1E464FEAF1427C
:1080B80082EA714282EA9122716A366853F8044F63
:1080C80031440A444FEAB44181EAF41181EAD40107
:1080D8000A449D42DA63E7D1036D0093436D01932F
:1080E800836D0293C36D0393036E0493436E0593EC
:1080F800836E0693DDE905ECC36E009CDFF8AC9057
:108108000793DDE90381DDE901659B4600274FEA16
:10811800F12383EAB11383EA716A59F827301A46C2
:1081280008AB53F827301A44134653442CEA01028B
:1081380001EA0E0A82EA0A021A444FEA743A86EA07
:1081480005035A448AEAB40A06EA050B234083EA7F
:108158000B038AEAB45A01379A44402F02EB08030A
:10816800E3465244A8461AD1009F1744019A07656E
:1081780022444265029A32448265039A2A44C265BF
:10818800049A1A44059B02660B444366069B734493
:108198008366079B6344C36649B0BDE8F08FF44625
:1081A80035468E46264619461446B0E7C4EF020007
:1081B80030B5E0B10F4A104900240025C0E9124546
:1081C800C0E914120D4C0E4A0E4DC0E916420E4A73
:1081D800C0E918520D4A826602F17452A2F52302D0
:1081E8000023A2F692420364C266184630BD0E20F0
:1081F800FCE700BF85AE67BB67E6096A72F36E3CB1
:108208003AF54FA57F520E518C68059BABD9831F59
:10821800F8B50446F0B10AB90020F8BDD1B10D4651
:108228008E180027B542F7D0236C15F8012BE254BD
:108238000133402B2364F5D121462046FFF71EFF6A
:10824800D4E9120110F5007241F10003C4E91223C8
:108258002764E7E70E20E0E72DE978480D46164643
:108268000446002800F08480002900F08180026C18
:108278008021372A02F1010381544FF000024DD8C2
:10828800382B46D1D4E91223206C0821E1FB0023C6
:1082980022FA01F1934684F83F2084F83E10110C2D
:1082A800120E84F83C201A0A9C4684F83B3084F865
:1082B8003A201A0C1B0E84F83D10C4E912BC214662
:1082C80084F8392084F838302046FFF7D7FE691E35
:1082D8007EB30023E26EDA4001F8012FA26EDA4085
:1082E8000A71626EDA400A72226EDA400A73E26D2F
:1082F800DA400A74A26DDA400A75626DDA400A76CD
:10830800226DDA400833202B0A77E3D10020BDE83C
:108318007888E2540133B3E7E25401333F2BFBD9A9
:1083280021462046FFF7AAFE3822002106F07AF8F7
:10833800A8E71823226DDA4001F8012F626DDA40B0
:108348000A71A26DDA400A72E26DDA400A73226E8F
:10835800DA400A74626EDA400A75A26EDA400A766A
:10836800E26EDA40083B13F1080F0A77E2D1CDE755
:108378000E20CCE7024AD2F80034002BFBD070471D
:1083880000E001400A4908B50223C1F80435BFF3EB
:108398006F8FBFF34F8FC1F80805FFF7EBFF00237E
:1083A800C1F80435BFF36F8FBFF34F8F08BD00BF0F
:1083B80000E001400E4B10B50124C3F80445BFF39B
:1083C8006F8FBFF34F8F01EB8204401AA14208D18F
:1083D800074B0022C3F80425BFF36F8FBFF34F8FFD
:1083E80010BD431851F8042B1A60FFF7C3FFEDE7DF
:1083F80000E0014043689B68184708B543680830A7
:108408005A7900F0DDFE002008BD2DE9F0430D4645
:108418009BB0084699469046FFF7ECFF6E68747962
:108428004C4528BF4C4607462246414602A800F064
:10843800ABFE727922990AA800F0C2FE00970AAB37
:10844800224602A905F1080001F0F0FD002848F2D3
:10845800425018BF00201BB0BDE8F0830023C0E9DC
:1084680002328B881A44B1F9063002611A44C0E915
:10847800001142610888003018BF01207047426827
:10848800118838B50346002937D0148A02F1100143
:1084980041602CB9C2680168FFF7E0FF204638BD8B
:1084A8009078118900F03005302D14D1947C04F0B7
:1084B8003004302C0FD190881969091A19610021EC
:1084C800908AB2F9162008441969014419611144C7
:1084D80059610120E3E700F0F004202C07D150890E
:1084E8004143002DECD1986801309860E8E700F02E
:1084F800C000802808BF0421F3E70846CFE770B51D
:10850800456804460E4663681A88B24204D19B78CF
:1085180003F00F03082B07D12046FFF7B0FF63686D
:10852800AB42F0D1002070BD0120FCE743681A443B
:10853800426011B101399A4201D10120704713F804
:10854800010B01F8010FF6E7836810B504460BB973
:10855800002010BD0368012298470028F8D0A368BE
:10856800013BA360F5E72DE9F3410F460DF1070143
:108578008046FFF7E9FF064620B90026304602B0DC
:10858800BDE8F0819DF80740220613D504F07F046A
:1085980007250DF107014046FFF7D6FF0028ECD06C
:1085A8009DF8072002F07F03AB401C43130605F13A
:1085B800070501D43C60E1E7232DEAD1DDE770B57A
:1085C8004568AA7802F00F06082E86B003461FD128
:1085D80003691C6800260CB906B070BD2368626880
:1085E8009D68267329466846FFF738FF6368049339
:1085F80004F10C030593AB7803F0C003802B08BF8C
:10860800231D684608BF0493FFF7D9FFA468E2E773
:1086180012F0C0011CD102F0300010280AD15A69AA
:108628001170072EEC68186909D10146204600F040
:1086380017F8D1E79006F4D55B691980CCE72A8949
:10864800214614B105F0C5FEC6E705F0EBFEC3E709
:108658008029C1D10069002192060160BCD5EBE7F1
:108668007FB50A4601466846FFF7F8FE30B168460E
:10867800FFF7A5FF6846FFF702FFF7E707B05DF8C9
:1086880004FB000030B5044685B01546A9B9026858
:10869800114B9A4211D0102D06D82A466946204619
:1086A800FFF7F0FF05B030BD102269462046FFF7FE
:1086B800E9FF0028F6D0103DEDE7A368AB4201D2F0
:1086C8000020EFE723682A46204698470028F7D07D
:1086D800A3685D1BA560E5E735850200F7B50E4682
:1086E80001A907461546FFF73EFFA8B1019A0123E5
:1086F800D3184FF0000404D2B17801F0C0018029EA
:1087080001D1204608E031899942FAD329463846F2
:10871800FFF7B8FF019BEC5403B0F0BD73B50E46EC
:1087280001A905461446FFF71EFFB8B1019BB3F532
:10873800803F07D202229A1804D2B17801F0C00112
:10874800802901D1002009E031899142FAD32146DC
:108758001A4621F8023B2846FFF794FF02B070BD85
:1087680010B5034C82600022C0E90041C26010BD10
:10877800358502002DE9F04F824685B00D464FF051
:1087880000084FF0000900240DF10F015046FFF7D3
:10879800DBFEF8B19DF80F1001F07F025FFA82FB53
:1087A8004FF0000CCDE900BC009AA4F1200CC4F1F4
:1087B800200322FA03F302FA0CF71F431346A340DF
:1087C80048EA03080B0649EA070904F1070404D438
:1087D800C5E9008905B0BDE8F08F462CD4D100204A
:1087E800F8E773B50D4669461446FFF7C3FF68B14D
:1087F8002B89082B0CD1DDE90056C4E90056DDE9C8
:108808000023B34206BFAA420120002002B070BD77
:10881800042B05D1DDE90001206005460026EEE7BE
:10882800022B03D10098208085B2F7E7012B05D1F0
:10883800DDE90001207000F0FF05EFE70020E5E723
:1088480037B50D4669461446FFF794FF30B12A89BB
:10885800082ADDE9003103D1C4E9003103B030BD95
:10886800042A18464FEAE37108D123601A460B46DA
:108878008B4206BF824201200020EFE7022A04D182
:108888001BB223801AB2D317F2E7012A03D15BB2D5
:1088980023705AB2F7E70020E0E7F7B50C4600214D
:1088A80019702170116001A9074615461E46FFF789
:1088B8005AFE30B9BB6813B901233370002003B0E6
:1088C800F0BD01990029F7D0CB0801F007012B6012
:1088D8002170F4E713B5044605291FD8DFE801F035
:1088E800030F151E1E1C012201A92046FFF7CAFE10
:1088F80018B19DF90430002BF5DB02B010BD082239
:1089080000212046FFF7BEFEF7E701A9FFF72BFE7F
:108918000028F2D0019AF3E70422F1E70020ECE7FF
:1089280073B50D4601A90446FFF71DFE064618B9A2
:108938000026304602B070BD94E80F0085E80F00AD
:1089480001998A42F4D3A960A3685B1AA360F0E78F
:108958002DE9F0415468A37813F0C00E88B006469C
:108968008C46154604D0BEF1400F68D0002444E080
:1089780003F00F025C4903F03003102B51F822700A
:108988001DD006D8002BF1D12A692146B8470446E4
:1089980033E0202B17D0302BE8D16B692188198060
:1089A800072A09D171462289286905F03BFD6B68C1
:1089B8002969D868FFF754FE2A6969683DE06B6940
:1089C80001221A70E0E7BCF1020FD5F8148027D114
:1089D800042A25D804A9FFF7A3FF04460028C5D018
:1089E800069B2BB16968B8F800304A899A4208D8C2
:1089F800059B7360069B002BB8D1204608B0BDE8E4
:108A0800F08108892A6903FB002204A8B84728B125
:108A1800B8F800300133A8F80030E1E70446E7E78A
:108A2800B8F800302969228903FB0212618999424A
:108A38009CD90133A8F8003021463046A6E71769CB
:108A48003B6807F1040813B9FFF744FF9FE70229C1
:108A580013D104A9FFF764FF002887D03B68696831
:108A6800424604A89847044600283FF47FAF069B77
:108A7800002BF3D1059B7360BFE701292BD009D3E5
:108A880005297FF473AF04220DEB0201FFF7FAFD0D
:108A9800042425E0002401AB191901340B2C3FF400
:108AA80065AF01223046FFF7EDFD00283FF45EAFC9
:108AB80001AB234413F9013C002BECDB0B4B049373
:108AC80001ABCDE905340023079342463B6869684A
:108AD80004A898475BE7082201A9FFF7D3FD0824FB
:108AE8000028EBD142E700BFD0F002003585020034
:108AF8002DE9F04F91B00446002604A8CDE902669E
:108B0800FFF7ACFCA3683BBBDDE9053404A89D78FE
:108B1800FFF7B5FC0028F7D115F0300F03D1059BFE
:108B28001B8803B10134002C00F0A98063090022DE
:108B380002A9934240F09C8010AA02EB830304F040
:108B48001F04C4F120044FF0FF3053F8383CE040D4
:108B5800C31A584258410DE00DF1030301AA0DF163
:108B680002012046FFF799FE38B99DF80330002B23
:108B7800CAD1002011B0BDE8F08F019904A8FFF711
:108B8800BEFC002850D1019BB3427FD3059D059AB6
:108B9800937803F00F03082B73D004A8FFF76FFC3A
:108BA800059B9D42F3D14FF0FF36019FB7426DD32D
:108BB800089B9DF80290D4F808801D684FF0010AC0
:108BC800A368002D5FD098459CD12B68D3F800B0DE
:108BD800BBF1000F08D04B463A4629462046D847F5
:108BE8000028C6D0AD68EBE7D3F808B0BBF8003072
:108BF8009F42F7D16A6859460AA8FFF72FFC6B68AD
:108C08000E9305F10C030F939BF8023003F0C00399
:108C1800802B04BF2B1D0E930AAA85F80CA0494689
:108C28002046FFF795FEDBE7059B9B7813F0300F96
:108C38000FD1069A3F2A0CD8510910AB03EB8101DA
:108C480002F01F020123934051F8382C134341F8D6
:108C5800383CE5689DF802201DB104AB0199204617
:108C6800A84704AA9DF802102046FFF771FE12E0FB
:108C780051F8225001357FF47DAF013259E70120C8
:108C880078E7168891E798457FF43CAF9DF8021085
:108C98002046FFF71FFE00287FF434AF69E770B560
:108CA8000C460646154611462046FFF7D9FC2A46CB
:108CB80021463046BDE87040FFF71ABFF0B585B0D1
:108CC8000C46CD68694607461646FFF729FE68B187
:108CD800E06858B1A37803F03003202B32462946C8
:108CE800684605D1FFF7DBFF019B7B6005B0F0BD4F
:108CF800FFF7FEFEF8E72DE977480E466946FFF7CD
:108D080039FD88B1DDE90023002502F001045FEA9E
:108D1800530C4FEA320B54EA050308D06FEA0B02F2
:108D28006FEA0C03C6E9002303B0BDE87088C6E902
:108D380000BCF9E737B50D4669461446FFF7DBFF77
:108D480068B12B89082B0CD1DDE90001C4E90001C9
:108D5800DDE900238B4206BF82420120002003B0D8
:108D680030BD042B03D100982060C117F0E7022B17
:108D780004D1BDF90000208000B2F6E7012B04D130
:108D88009DF90000207040B2EFE70020E7E713B537
:108D980004220C460DEB0201FFF774FC08B1019B9D
:108DA800236002B010BD1146FFF7F1BF13B50822CA
:108DB8000C466946FFF766FC18B1DDE90023C4E9F3
:108DC800002302B010BD1146FFF7F0BF02494FF46F
:108DD800F370FEF797B900BF39F10200022810B509
:108DE800044603D908494120FEF78CF9074B1C5D5E
:108DF8001F2C01D9FFF7EAFF01234FF0A042A3403F
:108E0800C2F80C3510BD00BFF4F0020036F10200C4
:108E1800022810B5044603D908494720FEF772F91D
:108E2800074B1C5D1F2C01D9FFF7D0FF01234FF022
:108E3800A042A340C2F8083510BD00BFF4F00200FC
:108E480036F1020008B50020FFF7E2FF0120FFF726
:108E5800DFFF0220BDE80840FFF7DABFC20710B500
:108E680004460AD54FF0A0430322C3F84427C3F8A9
:108E78004827C3F84027FFF7E5FFA3070AD54FF0B7
:108E8800A0430C22C3F83427C3F83827C3F83C277B
:108E9800C3F8402710BD000038B1054B0360054BEF
:108EA800436001230372002070470E20704700BF03
:108EB800E78E0200C18E020069B10B78022B0CD13B
:108EC800022804D003280CBF112008207047032370
:108ED8000B70002070470E2070470820704710B5AF
:108EE8000C4681B10B78042B04D8DFE803F00E059B
:108EF800030E0E00112010BD03F09EFE0028FAD1CB
:108F080002232370F7E70E20F5E70820F3E70000B7
:108F1800F8B5044680691649164A10F8025C521AD8
:108F28000C230E46B2FBF3F23DB9206953430022ED
:108F38009A4205D10123236013E04FF0FF30F5E793
:108F4800B758AF4201EB020E06EB020C0ED1471CDC
:108F580008D1DEF80850D4E90223D4E90001A84773
:108F68002060F8BDDCF804708742F2D00C32DFE7ED
:108F780040E502004CE502001EF0040F0CBFEFF3C1
:108F88000880EFF30980FFF7C3BF00BF28B139B1EC
:108F98000023C1E900301846704748F21050704766
:108FA80048F21350704730B1036848F240508B4282
:108FB80008BF0020704748F21050704728B148F2A7
:108FC8001150914208BF0020704748F21050704776
:108FD80070B506460C461D46FFF7D8FF50B9B37961
:108FE8004AB1AB420AD111462046FFF706FA08B942
:108FF800044B236070BD48F21050FBE748F2115053
:10900800F8E700BF7052464D2DE9F0470C46074679
:109018000F49204615469846DDE90869FFF7C3FF62
:1090280098B963685A79494652003046FFF7C6FF37
:1090380058B945B1089643462A4621463846BDE800
:10904800F047FFF7E2B948F21050BDE8F08700BFDB
:109058007052464D10B5044638B149B141600B68AD
:10906800984708B9044B236010BD48F20150FBE74C
:1090780048F21050F8E700BF6E524648F0B448B1C5
:1090880007680A4EB74209D159B16AB14368F0BCC2
:109098005B68184748F20150F0BC704748F202502C
:1090A800FAE748F21050F7E71046F5E76E524648DF
:1090B800F0B460B107680C4EB7420CD171B1436887
:1090C8001568DC68A5420CD39B68F0BC184748F2C9
:1090D8000150F0BC704748F20250FAE748F21350CA
:1090E800F7E748F21450F4E76E5246482DE9F0418C
:1090F800044617469846DDE90656FFF7ABFF60B908
:10910800424639462046FFF7B9FF30B9324629466C
:109118002046BDE8F041FFF7CBBFBDE8F081000075
:10912800F8B50A4F0A4C0B4DE41B0121E4082970DD
:109138000026A64203D102232B700020F8BD57F861
:10914800363098470028F9D10136F2E738E50200B1
:1091580038E502001C6C002038B50C46054618B9E5
:1091680008493320FDF7CEFF611E2944284688426E
:1091780000D938BD03780A7800F8012B01F80139C5
:10918800F5E700BF64F1020070B50D4614460646C7
:1091980018B90A494520FDF7B5FF1DB9074946200A
:1091A800FDF7B0FF621E3244013DB24200D270BDED
:1091B80015F8013F02F80139F7E700BF64F1020032
:1091C80070B5164604460D46FFF7DEFF3246A9196C
:1091D800A019BDE87040FFF7D7BF38B50D46044663
:1091E800FFF7BAFF29466019BDE83840FFF7B4BF5A
:1091F80008B507281BD8DFE800F004121A1A1A0469
:109208001A040120FFF72AFE0020FFF7E7FD0120DE
:10921800FFF7E4FD0220BDE80840FFF7F9BD012093
:10922800FFF7F6FD0220BDE80840FFF7D7BD08BDEF
:1092380008B5FDF7FFFCFDF79FFA0028FBD10D4D9F
:10924800642445F001054FF47A40A847013CFAD15F
:10925800094B1B68DB0700D500BEBFF34F8F0749DA
:10926800074BCA6802F4E0621343CB60BFF34F8F29
:1092780000BFFDE750F20200F0ED00E000ED00E075
:109288000400FA0507B5074B074C0092E41AE408F6
:1092980024040B460246054944F00100FDF712FC80
:1092A800FFF7C6FF4CE502004CE50200FCF10200A6
:1092B80008B5064A064B07499B1ADB081B040246F9
:1092C80043F00100FDF7EAFBFFF7B2FF4CE50200AF
:1092D8004CE5020033F202000022104638B54FF484
:1092E800805101F0AFFA024608B1FFF7E1FF1348D9
:1092F800C0F5FC2101F0A6FA01460028F5D1104876
:10930800104CFDF7DBF9FDF705F90F4B0F49E41A8F
:10931800E408240444F003042046FDF7BBFB0C4892
:1093280001F042F905460028DFD101F04DFA204648
:109338000849FDF7AFFB284638BD00BF00600200B2
:1093480009AC02004CE502004CE5020056F20200AE
:10935800F991020062F202008B1802448B4200D19C
:10936800704713F8010D02F8010DF7E7000000003F
:109378000000000000000000C3F10803DB0070B526
:109388000133002403A500BF5B1920C940CAAD19E9
:1093980020C0184720C940CA754120C020C940CA0A
:1093A800754120C020C940CA754120C020C940CAA3
:1093B800754120C020C940CA754120C020C940CA93
:1093C800754120C020C940CA754120C0644120466B
:1093D80070BD00BF00000000C3F10803DB0070B5DA
:1093E8000133002403A500BF5B1920C940CAAD1B87
:1093F80020C0184720C940CAB54120C020C940CA6A
:10940800B54120C020C940CAB54120C020C940CAC2
:10941800B54120C020C940CAB54120C020C940CAB2
:10942800B54120C020C940CAB54120C06441B4FA42
:1094380084F0400970BD00BF2DE9F04F08B4F8CAA8
:1094480004B451F8042BA3FB028940F8048B4FF0B5
:10945800000AE4FB629A4FF0000BE5FB62AB4FF0A9
:10946800000CE6FB62BC4FF0000EE7FB62CE51F841
:10947800042B4FF00008E3FB628940F8048BE4FBFF
:10948800629AE5FB62ABE6FB62BCE7FB62CE51F891
:10949800042B4FF00008E3FB628940F8048BE4FBDF
:1094A800629AE5FB62ABE6FB62BCE7FB62CE51F871
:1094B800042B4FF00008E3FB628940F8048BE4FBBF
:1094C800629AE5FB62ABE6FB62BCE7FB62CE51F851
:1094D800042B4FF00008E3FB628940F8048BE4FB9F
:1094E800629AE5FB62ABE6FB62BCE7FB62CE40F842
:1094F800049B40F804AB40F804BB40F804CB40F8A8
:1095080004EB0CBC052B00F01E810C68A0F11400C4
:10951800A1F11401A2F1140252F804EB4FF0000576
:1095280050F8046BE4FB6E5652F804EB50F8047BD9
:10953800E4FB6E6752F804EB50F8048BE4FB6E789A
:1095480052F804EB50F8049BE4FB6E8952F804EBE4
:1095580050F804ABE4FB6E9AA0F1140052F8044BE7
:1095680051F804EB4FF0000CE4FB6EC540F804CB57
:1095780051F804EBE4FB6E5640F8045B51F804EB39
:10958800E4FB6E6740F8046B51F804EBE4FB6E787B
:1095980040F8047B51F804EBE4FB6E8940F8048B37
:1095A80051F804EBE4FB6E9AA0E80006062B00F0E5
:1095B800CA800C68A0F11800A1F11801A2F11802E4
:1095C80052F804EB4FF0000550F8046BE4FB6E56BC
:1095D80052F804EB50F8047BE4FB6E6752F804EB96
:1095E80050F8048BE4FB6E7852F804EB50F8049BB7
:1095F800E4FB6E8952F804EB50F804ABE4FB6E9A76
:1096080052F804EB50F804BBE4FB6EABA0F1180071
:1096180052F8044B51F804EB4FF0000CE4FB6EC514
:1096280040F804CB51F804EBE4FB6E5640F8045BB9
:1096380051F804EBE4FB6E6740F8046B51F804EB57
:10964800E4FB6E7840F8047B51F804EBE4FB6E8988
:1096580040F8048B51F804EBE4FB6E9A40F8049B45
:1096680051F804EBE4FB6EABA0E8000C072B6AD0C2
:1096780008B40C68A0F11C00A1F11C01A2F11C02A5
:1096880052F804EB4FF0000550F8046BE4FB6E56FB
:1096980052F804EB50F8047BE4FB6E6752F804EBD5
:1096A80050F8048BE4FB6E7852F804EB50F8049BF6
:1096B800E4FB6E8952F804EB50F804ABE4FB6E9AB5
:1096C80052F804EB50F804BBE4FB6EAB52F804EB21
:1096D80050F804CBE4FB6EBCA0F11C0052F8044B1C
:1096E80051F804EB4FF00003E4FB6E3540F8043BFF
:1096F80051F804EBE4FB6E5640F8045B51F804EBB8
:10970800E4FB6E6740F8046B51F804EBE4FB6E78F9
:1097180040F8047B51F804EBE4FB6E8940F8048BB5
:1097280051F804EBE4FB6E9A40F8049B51F804EB03
:10973800E4FB6EAB40F804AB51F804EBE4FB6EBC01
:10974800A0E8001808BCBDE8F08F002310B51C463F
:109758005AB2914200DC10BD40F823400133F7E7CC
:1097680010B500231A465CB2A14203DCB2FA82F0BB
:10977800400910BD50F8234001332243F3E74A1152
:10978800012350F8220001F01F0103FA01F10840FB
:109798007047013949B2002904DA013149B231B9B7
:1097A8000846704750F82130002BF2D0F5E701F158
:1097B8008043013B50F82330002023B9013900EBE6
:1097C800411108B270475B080130F6E710B5002375
:1097D8005CB2A24200DC10BD51F8234040F823409F
:1097E8000133F5E710B5013A52B2002A01DA002038
:1097F80010BD13B250F8234051F823309C4203D8CF
:10980800F1D24FF0FF3010BD012010BD00EB8101F7
:109818000023884200D3704751F8042C43EA5203CE
:1098280041F8043DD307F4E770B59DF910401E4692
:1098380023460546FFF7A0FD30B9224629463046A3
:10984800FFF7D0FF012807D023463246294628468D
:10985800BDE87040FFF7C0BD70BD70B59DF9104000
:109868001E4623460546FFF7B7FD38B12346324664
:1098780029462846BDE87040FFF77EBD70BD2DE93A
:10988800F04FB5B004AD9DF9F8401F468046234619
:109898002846FFF7D1FD24AB2146384602930395AD
:1098A800FFF777FFC0EB841005B26B4203F01F038C
:1098B8004FF0200695FBF6F676B205F01F0914A8BE
:1098C80058BFC3F100093146FFF73FFFB9F1000F58
:1098D80030B22BDD14AB002203EB8000C9F1200E5F
:1098E8001346A34217D327B27B00019314AB03EBB3
:1098F800870704F1FF3934AB012603EB8909002DF2
:1099080055DB34AB0022C6F10100964603EB860A0C
:1099180003EB80002DE057F8236006FA09F10A43AB
:1099280040F8232026FA0EF20133DAE714AB224678
:10993800394603EB8000FFF749FFD4E70FFA81FCB3
:109948005AF8C83C53F82CB034AB03EB810151F8FA
:10995800803CABEB0303A3EB0E039B4504D034BF61
:109968004FF0010E4FF0000E50F8C81C41F82C3093
:109978000132019B51B29942E0DBA6EB0E035E4235
:10998800214614A85E41FFF741FF34AB03EB840383
:10999800214653F8802C59F8803C384643EAC27374
:1099A800013D49F8803C2DB2FFF730FFA7E734AB03
:1099B80003EB8606224656F8C81C4046FFF706FF0A
:1099C80035B0BDE8F08F30B51C4691B0054693F927
:1099D80000306846FFF730FDD4F8AC3069462846B9
:1099E800984711B030BD13460A46FFF7ECBF2DE982
:1099F800F04793F9006092B0044689461046314614
:109A080015469846FFF7ACFE002840F09380424682
:109A1800494602A8FFF7E7FF434602AA21460AA8DB
:109A2800FFF7D1FF02A908464246FFF7DCFF43468D
:109A38002A4649464846FFF7C6FF08F1040742464A
:109A480029462846FFF7CFFF3B462A4621462046AF
:109A58000096FFF7E9FE3B462A4629462846009627
:109A6800FFF7E2FE3B462A46214628460096FFF7C6
:109A7800F4FE43462A4621462046FFF7A4FF3B460C
:109A88002246214628460096FFF7CEFE3B46009622
:109A98002A4621462046FFF7C7FE2368DB074CD538
:109AA80033463A4621462046FFF766FC3146824651
:109AB8002046FFF7ABFE06F18043013B54F8230034
:109AC80040EACA7044F82300424621462846FFF778
:109AD8008AFF3B460AAA294628460096FFF7BDFE9C
:109AE8003B460AAA294628460096FFF7B6FE0AA969
:109AF80008463B462A460096FFF7AFFE43460AAAA9
:109B080021462046FFF75FFF02AA3B461046214642
:109B18000096FFF7A2FE324629462046FFF756FE7A
:109B2800324649462846FFF751FE324602A94846C2
:109B3800FFF74CFE12B0BDE8F08731462046FFF72C
:109B480065FEC1E72DE9F04115468AB0044688460E
:109B58002022002102A804F065FC2E1D95F9007052
:109B680003232A46414620460293FFF73CFF33462B
:109B780002AA214620460097FFF76FFE2B46424671
:109B880021462046FFF71FFF0097334605F1840260
:109B980021462046FFF748FE0AB0BDE8F0810000E4
:109BA800F0B5082289B00C460646FFF70FFECB6ACF
:109BB80003930B6B04934B6B05938B6B0693CB6BE7
:109BC8000793002708236A46694668460297019763
:109BD8000097FFF7D1FB082305466A463146304611
:109BE800FFF7CAFB236B0393636B0493A36B059383
:109BF800E36B0693054408236A4669466846079757
:109C0800FFF7BAFB082305446A4631463046FFF79A
:109C1800B3FB236A0093636A0193A36A0293A36B5D
:109C28000693E36B0793054408236A46314630469A
:109C3800059704970397FFF79FFB636A0093A36A4E
:109C48000193E36AA26B0293636B039304920693F6
:109C5800E26B236A0592054407936A460823314656
:109C68003046FFF789FBE36A0093236B0193636B2C
:109C78000293236A0693A36A0793054408236A4656
:109C880031463046059704970397FFF7A5FB236BEA
:109C98000093636B0193A36B0293E36B0393636A73
:109CA8000693E36A07932D1A08236A46314630461D
:109CB80005970497FFF790FB636B0093A36B0193E1
:109CC800E36B0293236A0393636A0493A36A05937D
:109CD800236B07932D1A08236A46314630460697A8
:109CE800FFF77AFBA36B0093E36B0193636A03931B
:109CF800A36A0493E36A0593636B07932D1A0823F9
:109D08006A463146304602970697FFF765FB2D1ADB
:109D18000D4C0FD435B9082231462046FFF762FDB5
:109D280001280FD00823224631463046FFF754FB5E
:109D38002D1AEFE70823224631463046FFF71CFB71
:109D48002D18F7D409B0F0BD74F20200F0B515462D
:109D580089B01C4607460E461A4629466846FFF74C
:109D680042FE23466A4639463846FFF72CFE23460C
:109D78002A4669466846FFF726FE23466A46314664
:109D88003046FFF720FE09B0F0BD2DE9F0438BB057
:109D98001446129D15F9046B00961F4680468946A5
:109DA8002B460246214602A8FFF757FD02A9129A40
:109DB8000846FFF718FE129B02AA41464046FFF7E5
:109DC80002FE129B02AA21462046FFF7FCFD2B4605
:109DD8004A46394638460096FFF73FFD129A3946FB
:109DE80002A8FFF700FE02A92B4642460846009645
:109DF800FFF733FD02A92B46224608460096FFF7D7
:109E08002CFD2B464246214620460096FFF725FDAD
:109E1800129B224649464846FFF7D5FD2B4602AA23
:109E2800414620460096FFF718FD129B2246394608
:109E38003846FFF7C8FD2B464A463946384600964D
:109E4800FFF70BFD324602A92046FFF7BFFC0BB017
:109E5800BDE8F0832DE9F047B3F9024088461E4675
:109E680004F11F012023073491FBF3F708234FFA6D
:109E780087F994FBF3F4944228BF144649460546F3
:109E8800FFF763FC22464146FFF766FAB6F902304F
:109E9800E4009C4221D9E41A05EB87010022C4F1B1
:109EA80020078D420FD324364A4629463046FFF70D
:109EB80099FC012811D04B46324629462846BDE870
:109EC800F047FFF789BA51F8040C20FA04F313435A
:109ED80041F8043D00FA07F2E3E7BDE8F08770B502
:109EE800036813F001050646144605D013460A46D2
:109EF8000146FFF741FA054621463046FFF786FC42
:109F080045B104F18042013A56F8223043F000434B
:109F180046F8223070BDF0B50F46A1B00646194686
:109F2800384615461C46FFF71BFC28B1214630462B
:109F3800FFF70BFC21B0F0BD224639466846FFF713
:109F480045FC2246294608A8FFF740FC214610A8F0
:109F5800FFF7FBFB0123214618A81093FFF7F5FB39
:109F6800224608A96846FFF73DFC28B9224610A9F1
:109F78003046FFF72BFCDDE7009BDA0709D42146C2
:109F88006846FFF743FC2246294610A8FFF7A7FFBB
:109F9800E6E7089BDB0707D4214608A8FFF736FC4D
:109FA8002246294618A8F1E7002823461CDD08AAFE
:109FB80069466846FFF710FA21466846FFF726FC0F
:109FC800224618A910A8FFF70DFC002805DA10A9E9
:109FD80023462A460846FFF7CFF910A9234618AAB0
:109FE8000846FFF7F9F9CEE708A96A460846FFF7D9
:109FF800F3F9214608A8FFF709FC224610A918A87A
:10A00800FFF7F0FB002805DA18A923462A46084678
:10A01800FFF7B2F918A9234610AA0846FFF7DCF99A
:10A02800BEE700000048704770F202002DE9F04FCB
:10A03800EDB01F46DDF8D8810590B8F9026098F9AF
:10A04800004020231F3696FBF3F676B206F1FF395F
:10A0580024AB002543F829506CAB03EB89034CA8CB
:10A068008A469346394698F9012043F8805C43F8BC
:10A07800605CFFF771F998F9012054A8B918FFF747
:10A088006BF921464CA8FFF76BFB0746002840F008
:10A098003981214654A8FFF763FB0290002840F05D
:10A0A800338108F1240332464CA918460393FFF77D
:10A0B80099FB012840F02A81324654A90398FFF7FA
:10A0C80091FB0128069040F021811CAD0CAF33466E
:10A0D800039A54A92846FFF71EFF029B47F8293028
:10A0E8005A46514638464346FFF7B4FE3946384685
:10A0F800039B00962A46FFF7C2FB0DF5B879039B30
:10A1080000962A464CA914A8FFF7B9FB48462246F0
:10A118000599FFF75BFBA30009EB030A0793059B6F
:10A12800A100591808F1440B50462246FFF74EFB90
:10A138005946224634A8FFF749FBA3000BEB03015D
:10A1480022463CA8FFF742FB08F10403494634AA1B
:10A15800284600940493FFF780FB53464A463CA9DF
:10A1680034A8CDF80080FFF710FE2346049A29464C
:10A178002846FFF7D0FE2A46514648464346FFF791
:10A18800E5FD029B08933146059B0A933846CDF8B6
:10A1980024B0CDF82C90FFF7FCFA3146814614A87C
:10A1A800FFF7F7FA8145B8BF81461FFA89F909F127
:10A1B800FF3B0FFA8BFB59463846FFF7E0FA594642
:10A1C800071C14A818BF0127FFF7D9FA002814BFE5
:10A1D800022300231F430DF1200A22465AF8277054
:10A1E80024A83946FFF7F2FA0DF1B00BA300F918CD
:10A1F80022465846FFF7EAFA21462846FFF7A5FA0D
:10A20800A9F10209069B2B600FFA89F90DF1900A52
:10A21800B9F1000F23DA2346049A29462846FFF7A6
:10A228007AFE43462A4659465046FFF78FFD324686
:10A2380051460398FFF7D6FA012805D03346039A0A
:10A2480051465046FFF7C8F8013C64B2002C4CDA7E
:10A25800029BB3FA83F040096DB0BDE8F08F434626
:10A268002A46D8F8A47059465046B84749460CA81B
:10A27800FFF785FA4946071C14A818BF0127FFF7FE
:10A288007EFA002814BF02200020384308AB53F898
:10A2980020702FB32246394634A8FFF797FA079B58
:10A2A8002246F9183CA8FFF791FA43462A463CA9EA
:10A2B80034A8FFF74BFD049B009434AA514644A8E8
:10A2C800FFF7CBFA5B4652463CA934A8CDF800808C
:10A2D800FFF75BFD434644AA29462846FFF773FB70
:10A2E80009F1FF390FFA89F992E723B26CAA02EB58
:10A2F80083025AF8233052F8802C5340029A1A43AA
:10A308000292A1E72846A7E73846A5E70298A3E7FF
:10A318000369C1688B429DBF8268D21802F1FF327F
:10A3280003F1FF3394BF501A581A70472DE9F041D2
:10A33800D0E902670446F61B4068964288461546EF
:10A34800384405D904F045F83D44E560BDE8F0819E
:10A358003246AD1B04F03DF82A4608EB060160685A
:10A3680004F037F8F1E72DE9F843C5680646894651
:10A3780017464FF000083469B3687068A54228BFD3
:10A38800E418013C621B5C1BBC4228BF3C4694425B
:10A3980028BF144649462844224604F01AF8B368F0
:10A3A8002544AB4208BF00253F1BA044A144F560EB
:10A3B800E1D14046BDE8F88310B5114C114AA261BD
:10A3C8000223C4E90433104BE361A2644FF48053C1
:10A3D8000E4A2362E264002310220D49A362E01DA5
:10A3E8006362E362A3656365E365226504F04DF883
:10A3F8000849204604F049F82023A37110BD00BF86
:10A40800206C002020F30200A86C0020986C00202B
:10A4180029F302002DF30200F8B5184C182300FBAD
:10A42800033503FB00402544C46A012C0F46164639
:10A4380011D003D3022C1BD000240AE02846FFF7D2
:10A4480067FF864205D8324639462846FFF76EFF31
:10A4580034462046F8BD2846FFF75AFF8642344660
:10A4680028BF0446224639462846FFF75FFFF0E733
:10A478002846BDE8F840FFF776BF00BF206C0020F3
:10A48800FFF79ABF41DF7047014B01221A707047EE
:10A49800C880002008B50948094B0A49C01AC008F5
:10A4A800000440F00400FCF7F5FA074B07480022C7
:10A4B8001A70BDE8084002F0C1BA00BF4CE50200BE
:10A4C8004CE5020034F30200C880002041A50200D8
:10A4D80008B50748074B0849C01AC008000440F0EF
:10A4E8000300FCF7D7FABDE80840FFF7D3BF00BF69
:10A4F8004CE502004CE5020056F30200C31E10B5FD
:10A508000446042B09D8DFE803F00303080F0F0003
:10A5180007494FF4701000F033FB064B1B6833B14A
:10A528002046BDE810401847FFF7B4FFF5E710BD17
:10A53800D9A40200CC80002008B5FCF77BFBFCF70F
:10A548001BF90028FBD10B4D642445F001054FF49D
:10A558007A40A847013CFAD1BFF34F8F0649074B11
:10A56800CA6802F4E0621343CB60BFF34F8F00BFA9
:10A57800FDE700BF50F3020000ED00E00400FA051B
:10A5880008B50648064B0749C01AC008000440F041
:10A598000400FCF77FFA002008BD00BF4CE502006C
:10A5A8004CE5020003F50200F8B56F4B6F4C70499B
:10A5B800E41AE408240444F0040705463846FCF786
:10A5C80069FA6C4B00201D6002F04EFA064640B94D
:10A5D80000F092FC012800F0BB8004D3022800F0B0
:10A5E800BF800320F8BD4FF08043D3F8005415F422
:10A5F800803551D04FF48032C3F8002435465E4E82
:10A60800336A012B5BD05D4944F00300FCF742FA42
:10A618005B493846FCF73EFA4FF4701400F098FD99
:10A62800584A20211820FCF735FC08B1FEF740FEF7
:10A63800554B1A6802F0F802B02A06D11A68D207F8
:10A6480042BF1A6802F04E021A604B4B9A6D012AFB
:10A6580006D10020986502F095F908B1FEF728FEAA
:10A66800FFF78EFF0028BCD12046484900F088FA41
:10A67800474800F051FF0028B3D146493846FCF757
:10A6880009FA00F0ABFDFCF78FFCFCF775F8002821
:10A69800F7D1FFF7F7FEF4E7D3F8202502F0F80228
:10A6A800A82A0AD1D3F82025D10706D5D3F8202522
:10A6B80002F05602C3F82025A1E701259FE743F2DF
:10A6C80004031A68344B9A420FD11DB996F86032C8
:10A6D800012B0AD0726B31484FF4805103F0D6F841
:10A6E80018B92F4944F0020090E702F083FB0146B5
:10A6F8001DB996F8A132012B06D0B269294803F09A
:10A70800C5F808B92849EDE728493846FCF7C2F9E1
:10A718001D4B1B6813F0B10F01D0254979E7B36DC4
:10A72800012B01D1234974E702F0BEFA00287FF417
:10A7380058AF214D2870214802F080F92B7823B9B1
:10A748001F494FF4FE70FCF7DDFC00F03DF801E016
:10A75800FFF7A0FE1B4944F00100FCF79BF940E716
:10A768004FF4A0245AE700BF4CE502004CE5020074
:10A778006AF30200CC8000209C98002081F302003C
:10A788001FF40200A87C00201C050040D9A4020088
:10A7980005A502009BF40200DBE5B151FC9A0020FC
:10A7A800AFF302003D9B0020EAF3020012F402001E
:10A7B80042F4020063F40200C880002091A4020061
:10A7C800ABF402008FF4020070B5184B184C194D09
:10A7D8001949E41AE408240444F004064FF48052AA
:10A7E8003046FCF75BF9D5F8802014493046FCF771
:10A7F80055F94FF0FF33C5F88030C5F88031C5F8FA
:10A808008430C5F8843101F086FD20B10C4944F04C
:10A818000100FCF73FF9FBF7AFFF0028FBD14FF42D
:10A828008050BDE8704000F039B800BF4CE5020028
:10A838004CE5020000E100E01DF5020053F50200BE
:10A848007DF50200C1F30B0330B52BBBB0F5FE2F2D
:10A8580022D8000B013900EB113101254FF080425D
:10A86800814201D2002030BD00F01F03440905FADF
:10A8780003F3032C05D8DFE804F00206090CC2F83C
:10A8880000360130ECE7C2F80436FAE7C2F81036B1
:10A89800F7E7C2F81436F4E70720E4E730B50446D2
:10A8A8002C48002289B0C0F5FE21FFF7CBFF0246F5
:10A8B80048B12948294B2A491B1ADB081B0443F0D5
:10A8C8000100FCF7EBF802F095FA264B9969002293
:10A8D80001441046FFF7B6FF024648B11E481F4B19
:10A8E80021491B1ADB081B0443F00100FCF7D6F8CA
:10A8F800EFF305810023D4E9002083F3148883F360
:10A90800108883F3118883F31388C1F3080139B9D8
:10A9180082F308884FF0FF339E46004709B030BDE8
:10A92800A2F120044FF0FF35CDE90033CDE9023321
:10A938000493CDE905504FF08073202269462046E4
:10A94800079303F046FD84F30888AE466FF00603CC
:10A958001847E3E7006002004CE502004CE50200FE
:10A96800B2F502009C980020E9F50200F7B5264BE5
:10A9780006462648C01AC00800040C463246244938
:10A9880040F00400FCF78AF8B4F1807F37D32149FE
:10A998008F20FCF7B7FB6FF07F431F4FA34228BF00
:10A9A8002346D7F80455E41A1D44631E942B96BF1A
:10A9B800963474607460347B25F07F4598BF963D6B
:10A9C800032C03D913497720FCF79CFB04F5A873E3
:10A9D800124A47F823504FF4F86042F001029047BA
:10A9E8000F4BA200134400221A601B680193019BBD
:10A9F8004FF48033A340C7F8043303B0F0BD952C5F
:10AA0800C9D804499020C4E74CE502004CE502008F
:10AA180056F602006CF602000040024050F60200B2
:10AA28004041024018490A7884B0002A29D14FF0E1
:10AA38008043A020D3F81834DB035EBF134B0122F8
:10AA48001A60134A0023136012680392039A114A8A
:10AA5800136012680292029A0F4A136012680192F8
:10AA6800019A0E4A82F82403102050600C4A0D48BF
:10AA7800C2F808350123036002201360C2F80403FA
:10AA88000B7004B0704700BFD4800020080000405D
:10AA980000410240404102404441024000E100E0E0
:10AAA80000400240084002402B4B2DE9F7431A684A
:10AAB80042B12A490A6801320A6000221A601B68FA
:10AAC8000093009B2648274BDFF8B080264EC01A1B
:10AAD800C0080004A8F5102740F00405A7F5A067F2
:10AAE800336823B300233360B4003368019307EB62
:10AAF800040944444A461D49019B2846A4F51024EC
:10AB0800FBF7CCFFA4F2F44319491A784FF48033C9
:10AB18009340184A2846C2F808334A46FBF7BEFF56
:10AB2800A4F2FC43196849B14846FFF71FFF124BCE
:10AB380004369E42D4D103B0BDE8F083A4F59F63E8
:10AB4800196811B14846FFF711FFA4F5A0642368FE
:10AB5800002BECD09847EAE704410240D08000205F
:10AB68004CE502004CE50200404102401DF602009F
:10AB78002FF602000040024048410240D45700200E
:10AB8800F8B5114B114E044611483768C01AC00871
:10AB980000043A460D4640F004000E49FBF77EFFDC
:10ABA8003A7B4FF4803393400B4AC2F808334CB1D8
:10ABB8003668FFF737FF356021463046BDE8F84074
:10ABC800FFF7D4BEF8BD00BF4CE50200F4570020E3
:10ABD8004CE502001DF602000040024070B5074B2C
:10ABE8001C6805460E46A060FFF71CFF2660294634
:10ABF8002046BDE87040FFF7B9BE00BFF8570020F7
:10AC0800034A044B1068D3F8043503EB006070471F
:10AC1800D080002000400240014B01221A7070478A
:10AC2800D58000202DE9F341284FFA6A7E6ABC6C72
:10AC3800AC2A22D17B6B1C44F61A254B254D009675
:10AC4800ED1AED082D0445F004082346224A23494D
:10AC58004046FBF737FFFB6AAC2B14D0324621463F
:10AC68001D4803F080FBB8B91D494046FBF712FFA9
:10AC78000024204602B0BDE8F081002CDDD102F0AE
:10AC8800CFF80446D9E73246A4F58041124803F0CC
:10AC98006AFB0028E8D0E1E73346224611494046DE
:10ACA800FBF706FFFBF768FD0028FBD100F096FADA
:10ACB8002046314601F010FB04460028D9D00A4945
:10ACC80045F00100FBF7E6FED3E700BF9C980020A3
:10ACD8004CE502004CE5020000600200CFF60200DD
:10ACE80031F7020004F7020068F702002DE9F04F7F
:10ACF8003A4B17463A4A9B1A87B0DB081B04049361
:10AD0800814243F0040305468946039308D1354937
:10AD18001846FBF7BFFE0024204607B0BDE8F08FB9
:10AD280003D231494F20FCF7EDF9C5F30B031BB1F2
:10AD38002D495120FCF7E6F9A9EB05035FEA133B1F
:10AD480003D129495420FCF7DDF900F001FABBF1E1
:10AD5800080F28BF4FF0080B07F6FF784FEA0B33B0
:10AD68004FEA183805930FB93C46D5E7C34534BFB9
:10AD7800DA46C2464FF000025146284634BF059EC7
:10AD88003E4601F063FA04460028C5D12B464A46E0
:10AD9800164903980096FBF795FEF21C234622F00D
:10ADA80003024946284601F013FA04460028B3D1A5
:10ADB8000F4A136BBF1B3544B1441E44166301F0A0
:10ADC80043FEA8EB0A0804460028CCD0049B094996
:10ADD80043F00100FBF75EFE9EE700BF4CE5020072
:10ADE8004CE5020082F7020091F70200F7F7020033
:10ADF8009C98002018F802002DE9F04702F020F88E
:10AE0800344C354BDFF8ECA03449DAF84850DAF81E
:10AE18003080DAF83460E41AE408240444F00407C3
:10AE280081463846FBF736FE42F20403EA5803F13E
:10AE3800A34303F5471303F2D7539A4208D028498E
:10AE480044F00100FBF726FE03252846BDE8F087FD
:10AE5800DAF83020B242154405D122493846FBF7CA
:10AE680019FE0025F1E7DAB94FF4405338461B784C
:10AE7800142B81BF43F214031A681B4BB2FBF3F285
:10AE880005F500531B78142B81BF42F214031649B1
:10AE9800EB58B3FBF1F398BF00231449FBF708FE06
:10AEA800A6EB080202F6FF7222F47F62294622F01E
:10AEB8000F0209EB0800FFF719FF054628B10C49F6
:10AEC80044F00100FBF7E6FDBFE7BDE8F04701F0FD
:10AED800BBBD00BF4CE502004CE502001EFA0200B3
:10AEE80043FA020077FA020040420F0089FA020092
:10AEF800B2FA02009C9800202DE9F0475C4B5D4CAB
:10AF08005D4F5E49E41AE408240444F0040840460E
:10AF1800FBF7C0FDFB6AA52B00F0858009D8012B43
:10AF280020D044F003005649FBF7B4FD0020BDE8EB
:10AF3800F087AA2B00F08280AC2BF2D15149404611
:10AF4800FBF7A8FD50494046FBF7A4FDFFF754FF67
:10AF5800054600287BD04D4944F00100FBF79AFDD7
:10AF6800012620E04A494046FBF794FD7E6AD7F85F
:10AF7800489001F03FFF3D6B464900EB050A40460B
:10AF8800FBF788FD396B49448A4514BF721B0022C0
:10AF98005046FFF7ABFE054668B13F4944F0010053
:10AFA800FBF778FD0026FB6A3C492A4644F001007D
:10AFB800FBF77EFD12E001F01DFF2A463146FCF743
:10AFC80083F8BA6A9042814626D135494046FBF754
:10AFD80061FD0123C7E90793BE612E463148324D12
:10AFE80001F0FCFE002331482B7001F02DFD2B7879
:10AFF800814623B92E494FF4D170FCF783F8B9F193
:10B00800000F2CD196B33B6A012B2FD1404629491A
:10B01800FBF740FD02208AE70346274944F0010078
:10B02800FBF746FDD9E725494046FBF733FDFFF717
:10B03800E3FE01260546002DD0D0B4E7204940465E
:10B04800FBF728FDFFF7EEFD00260546F3E7FFF7BF
:10B05800E9FD054608B11B497EE70126BEE744F035
:10B0680001001949FBF716FD032060E701205EE7A0
:10B078004CE502004CE502009C98002051F80200C3
:10B088005DF9020006F9020014F9020031F9020024
:10B0980072F802007CF80200B2FA020076F90200A7
:10B0A80097F80200C0980020D580002021AC02004B
:10B0B80091F70200A8F90200ACF80200F4F80200C7
:10B0C800FDF8020047F9020004FA02000A4AD2F821
:10B0D80000347BB109480023D2F80815D940C907C4
:10B0E80048BF03F5C07103F1010348BF42F82100CE
:10B0F800072BF1D1704700BF000001403546526E62
:10B1080008B50748074B0849C01AC008000440F0B2
:10B118000300FBF7BFFCBDE80840FFF7D7BF00BF3F
:10B128005CE502004CE502003CFB020007B5074B5A
:10B1380000221A601B680193019BFBF77BFDFBF75C
:10B148001BFB0028FBD103B05DF804FB00010140A4
:10B1580070B5194E33784BBB184C1949194B641A02
:10B16800E408D3F80024240444F00304FAB1D3F823
:10B17800045515492A462046FBF790FC40F616531D
:10B188009D42B8BF1D46A5F54865FFF79FFF2A46B3
:10B198000E492046FBF782FC0D492846FFF71EFDA5
:10B1A8000C4B4FF480321A600123337070BD0A498A
:10B1B8002046FBF76FFCF7E7D68000205CE502002D
:10B1C8004CE5020000000140CBFA0200E4FA02005C
:10B1D80009B1020000E100E016FB0200034BD3F8BE
:10B1E80000340BB1FFF772BF704700BF0000014089
:10B1F8000C4B1B78062B10D10B4B1B681A070CD174
:10B208000A4B186800F0F003302B08D000F0E0007B
:10B21800A0F1400358425841704700207047012070
:10B22800704700BFE00F00F0E40F00F0E80F00F0F7
:10B23800094B1B78062B0CD1084B1B681A0708D141
:10B24800074B186800F0F000A0F13003584258414D
:10B2580070470020704700BFE00F00F0E40F00F0D7
:10B26800E80F00F008B5FFF7C3FF28B17D4B7E4A11
:10B278001B68C3F304231360FFF7DAFF10B17B4B9D
:10B288007B4A1A60FFF7B4FF28B17A4B7A4A1B68E9
:10B29800C3F342331360FFF7CBFF20B1774AD3687B
:10B2A80023F08073D360FFF7A3FF40B14FF08043D2
:10B2B8000022C3F80C21C3F81021C3F83825FFF782
:10B2C800B7FF10B16E4B03221A60FFF7B1FF40B110
:10B2D8006C4B05221A6001229A6700229A603F226D
:10B2E8005A60694B1B78062B50D1684B1B681907AD
:10B2F8004CD1674B1B6803F0F003502B46D14FF03D
:10B308008052644BD2F80414C3F82015D2F80814FC
:10B31800C3F82415D2F80C14C3F82815D2F8101461
:10B32800C3F82C15D2F81414C3F83015D2F8181431
:10B33800C3F83415D2F81C14C3F84015D2F82014F9
:10B34800C3F84415D2F82414C3F84815D2F82814C1
:10B35800C3F84C15D2F82C14C3F85015D2F8301491
:10B36800C3F85415D2F83414C3F86015D2F8381459
:10B37800C3F86415D2F83C14C3F86815D2F8401421
:10B38800C3F86C15D2F84424C3F87025FFF730FFD2
:10B3980028B1414B414A1B6803F04F031360FFF784
:10B3A80027FF48B14FF08043D3F80024D20744BFA9
:10B3B8006FF00102C3F80024394B1B68062B08D133
:10B3C800384B1B68062B01BF374A136843F4806368
:10B3D8001360364AD2F8883043F47003C2F88830D4
:10B3E800BFF34F8FBFF36F8F4FF01023D3F80022B6
:10B3F800002A03DBD3F80432002B2FDA2C4B01226E
:10B40800C3F80425D3F80024002AFBD04FF01022FB
:10B418001521C2F80012D3F80024002AFBD04FF0FF
:10B4280010231522C3F80422214B1A46D3F800141E
:10B438000029FBD00021C3F80415D2F80034002BF2
:10B44800FBD0BFF34F8F19491A4BCA6802F4E06268
:10B458001343CB60BFF34F8F00BFFDE7164B174A6E
:10B468001A6008BD240300104035014074C007402D
:10B478000DF0ADBA440200103C050040F0ED00E0CC
:10B48800A005004010560040E00F00F0E40F00F067
:10B49800E80F00F000C0004058020010E40E004021
:10B4A80030010010340100103C17004000ED00E0AE
:10B4B80000E001400400FA05FC5700200090D0038A
:10B4C80013681F2B10B5144607D900220830FCF763
:10B4D800C3FE08B92023236010BD48F21450FBE7CF
:10B4E8000830FCF795BE0830FCF762BE007800F023
:10B4F80001007047062810B5044602D1002001F06B
:10B5080033FC044B1B681BB12046BDE810401847AC
:10B5180010BD00BFD880002038B5104B104C186003
:10B52800104B1149E41AE408240444F00300FBF723
:10B53800B1FA0020FFF7DEFF0C4801F0DDFB0546FD
:10B5480020B90A48BDE8384001F098B902460849D0
:10B5580044F00100FBF7A2FA284638BDD880002045
:10B568004CE502004CE5020018FD0200FDB40200A3
:10B578002BFD02006CDF70476DDF704772DF70478C
:10B5880073DF704774DF704775DF704776DF704789
:10B598007ADF70477CDF70477DDF70477FDF704759
:10B5A80086DF70478FDF704790DF7047A8DF7047EE
:10B5B800AADF7047ADDF7047AEDF7047B0DF704776
:10B5C800B1DF7047B5DF704762DF704766DF7047ED
:10B5D80013DF70477FB50023CDF80A30ADF80E3081
:10B5E8000A4BADF806109B89ADF8083001238DF899
:10B5F8000A300DF10603CDE90430054B02A918887D
:10B60800FFF7DAFF07B05DF804FB00BF46910020A2
:10B618000258002010B5094B094904460948C01AC8
:10B62800C0080004224640F00400FBF737FA214620
:10B638000548BDE81040FBF7DFBE00BF4CE502003F
:10B648009E02030064E50200D0E5020070B5204EBA
:10B65800346814F0010432D01E4B984236D01E4B89
:10B668001E4D1F4C1F49ED1AED082D0445F0040529
:10B678002846FBF70FFA22884FF6FF739A4220D02C
:10B6880019492846FBF706FA3368208843F0040373
:10B6980013213360FFF77AFF044680B9134EC8249C
:10B6A80046F001064FF47A40B047013CFAD102F067
:10B6B80029FC044618B90E492846FBF7EBF9204641
:10B6C80070BD0C4B1878FFF75DFFF0E70024F6E734
:10B6D8007C91002038E502004CE5020064E5020098
:10B6E80002580020F8FD020015FE02009002030037
:10B6F80024FE02000058002030B518228DB00DEB52
:10B708000200002102F08EFE282308932448254BCE
:10B718002549C01AC0080004012440F004008DF82F
:10B7280018408DF82D40FBF7B5F91623ADF8063013
:10B738000023CDF80E30CDF81230ADF816301B4B83
:10B7480002930222062109251A7099701A710321A1
:10B758005922D9705A710DF10601FE225819ADF817
:10B768000C505C709A71FFF717FFB8B9BDF8062046
:10B778001D721119D971BDF80C301A440C4BADF873
:10B788000C2002A906AA1846FFF7F8FE30B9187867
:10B79800FFF7F8FE21461878FFF7F2FE0DB030BD2E
:10B7A80064E502004CE5020065FD02005A910020A4
:10B7B80000580020F0B50388212B8DB0044600F016
:10B7C8006A8132D8122B00F0398107D8102B56D055
:10B7D80075D8012B00F0AA810DB0F0BD142B00F034
:10B7E8003982C0F001811A2B00F045821F2BF3D15A
:10B7F800B24BB34DB349ED1AED082D0445F00400E2
:10B80800FBF748F9B04B04F108011888FFF7BCFEB4
:10B8180004460028E0D00246AC4945F00100FBF799
:10B828003DF92046FDF744FDD6E7502B5CD013D8F0
:10B83800232B00F0C780C0F01F81242BCCD19F4B55
:10B848009F486289A249C01AC0080004E38940F0F1
:10B858000400FBF72DF9BFE7522B00F00C82C0F073
:10B868006B81552B00F08280562BB5D18379002B44
:10B87800B2D1954B13211888FFF788FE9AE08F4BB9
:10B888008F4D9449ED1AED082D0445F00400FBF79F
:10B8980001F98D4BA2881A808F4A12681C460AB19A
:10B8A800012090478D492088FFF76EFE0246002848
:10B8B80092D08B4945F00100FBF7F0F88CE7824BFA
:10B8C8004FF6FF721A80874B1B685A0704D4FFF79C
:10B8D80013FF08B1FDF7ECFC7F4B1B68002B3FF40E
:10B8E8007BAF0220984777E77F4FC288BB889A4290
:10B8F8007FF472AF7D48724DFBF752FD6F4BED1A26
:10B90800ED082D04064628B9794945F00200FBF7F1
:10B91800C1F861E7F422238A76490092024645F08D
:10B928000400FBF7CFF8228A04F11201304602F036
:10B9380050FD182200210DEB020002F073FD0823D0
:10B948008DF818306C4B08936C4B0797CDE9093686
:10B9580006A8238AADF82C3000F070FF00283FF4C9
:10B968003BAF31466148FBF747FD35E7C288F62A09
:10B9780024D8D31E9B0723D0D31F9BB2013B594227
:10B9880001F0030103F0030302F1FF3458BF4B42F7
:10B99800E31A9CB2494B4A485949C01AC0080004E6
:10B9A800234640F00400FBF783F8474B21461888EC
:10B9B800FFF708FE00283FF40FAF33E7F724E9E765
:10B9C8001446E7E73D4B3E484E49C01AC0080004FC
:10B9D80040F00400FBF75EF8002206A9A088CDE934
:10B9E8000622FFF7E1FDE5E7344B354C4649364D75
:10B9F800E41AE408240444F004042046FBF74AF857
:10BA08000023ADF81A300223ADF8183006AA04ABAB
:10BA180042F6052128880793FFF7CCFD08B1FDF70A
:10BA280047FCBDF8102039492046FBF737F80023BA
:10BA38001A4685212888FFF7B1FDBBE71F4B204D2B
:10BA48003349ED1AED082D0445F004052846FBF7A7
:10BA580021F862892F492846FBF720F822892E49C8
:10BA68002846FBF71BF8A2892C492846FBF716F84D
:10BA7800E2892B4928461FE7437A827A0F49104802
:10BA8800401AC008217A00910004264940F00400B9
:10BA9800FBF718F8A0E6094B09482349C01AC00863
:10BAA800000440F00400FAF7F5FF0CA9002321F880
:10BAB800183DA088FFF776FD7CE700BF4CE5020043
:10BAC80064E502003201030002580020610103000E
:10BAD8002F00030041FF020080910020960203001E
:10BAE8004BFF02007C91002046910020D0E5020027
:10BAF80079FF020098FF0200D5BC02001DB60200C3
:10BB0800B8FF0200FEFF02006D000300950003006D
:10BB1800B8000300DF000300F50003000B01030079
:10BB28001D01030096010300D00103005B4B0021B7
:10BB38001888FFF74BFD3DE78379002B3FF44CAEA7
:10BB4800022B7FF449AE564D0289AB899A427FF4A5
:10BB580043AE837B012B7FF43FAE00230121CDE967
:10BB680006338DF81E10018AADF820104B4E418A1D
:10BB7800ADF82210022200F114018DF81820099165
:10BB8800ADF81230ADF8102003AB298A3088059340
:10BB980004AAFFF70FFD374660B91846FFF7A6FC61
:10BBA80040B940F2FD1306A93088ADF81C30FFF704
:10BBB80005FD11E6002306A93888ADF81C30FFF70B
:10BBC800FDFC014600287FF407AE18220DEB0200A9
:10BBD80002F028FC237D334A8DF81830022B079594
:10BBE800089224D0062B10D0012B10D12E4B1A8886
:10BBF8002E4B1A80637DD4F816200A93012B0B92E2
:10BC080005D12B4801F0B0F801E0637D0A9306A83E
:10BC180000F014FE024600283FF4DEAD2548264B0E
:10BC280026491B1ADB081B0443F0010044E6214B9C
:10BC380021482349C01AC008000440F00400FAF75C
:10BC480029FFA27D637D43EA0223174A1380174A1E
:10BC58001380DCE7174B18481A49C01AC0080004BB
:10BC680040F00400FAF716FF00231A461946A08888
:10BC7800FFF796FC9EE600231A461946A088FFF7B0
:10BC88009FFC08B1FDF714FB0B480A4B0E49C01A7C
:10BC9800C008000440F0040039E600BF0258002044
:10BCA80046910020D5BC0200849100208691002096
:10BCB80038E502004CE5020064E502000B020300CF
:10BCC800F90103003F0203006502030030B50D4689
:10BCD80087B0044620B9464940F28710FBF712FAAC
:10BCE80025B943494FF4C470FBF70CFA112200211F
:10BCF80001A802F097FB2378082B0BD13D4A3E4957
:10BD080013880988013B9BB2138031B32BBB0323F3
:10BD180011802370637822788DF805206021012B2B
:10BD28008DF804108DF8063019D034493448401A7B
:10BD3800C0080004334940F00200FAF7B9FE6378FE
:10BD48000B2B52D100F0BEFA8DF80700002000F04E
:10BD5800B3FA042101A8FFF73DFC07B030BD062A5D
:10BD68001DD0082A01D0032A3FD1D4E90123110AA2
:10BD78008DF807208DF80810110C120E8DF80A2086
:10BD88001A0A8DF80B308DF80C201A0C1B0E8DF842
:10BD980009108DF80D208DF80E300B21DAE7E168D7
:10BDA8008DF80710D4E90123080A8DF80800080C5B
:10BDB800090E8DF80A10110A8DF80B208DF80C1059
:10BDC800110C120E8DF80E201A0A8DF80F308DF80E
:10BDD80010201A0C1B0E8DF80D108DF809008DF827
:10BDE80011208DF812300F21B4E70321B2E700BF0C
:10BDF80074FD020086910020849100204CE5020029
:10BE080064E50200D1FD02002DE9F043804695B0BB
:10BE180020B9504940F24F40FBF774F94E4B4FF6AA
:10BE2800FF7214A91A804FF65963012021F8483D82
:10BE380042468DF80A00FFF7B9FB0446002840F097
:10BE48008580464B04AA03F1100615461868596800
:10BE5800144603C40833B3422246F7D108F102015D
:10BE68002846FFF7B1FB044600286FD101461C2283
:10BE78000DA802F0D7FA9DF83430ADF8044043F02D
:10BE880004038DF834300223ADF80C3098F80230F2
:10BE98008DF80E304FF00109C4F3072369F303034B
:10BEA80069F307138DF80530E3B243EA090369F330
:10BEB80042038DF80630F423CDE90A4401ADADF80C
:10BEC8002C3003AE08F1040308AA0DA9B8F8000045
:10BED8000C94CDE90865FFF76BFB27460446A8BB21
:10BEE80001461C220DA802F09DFA9DF83430ADF8E9
:10BEF800044043F018038DF8343098F802308DF878
:10BF08000E30C4F3072369F3030369F307138DF8AD
:10BF18000530FBB243EA090369F34203DBB243F09D
:10BF280010038DF806301723CDE90A4408AAADF8A6
:10BF38002C300DA908F10C03B8F800000C94ADF8EA
:10BF48000C90CDE90865FFF733FB0446204615B091
:10BF5800BDE8F08374FD02000258002055FD020080
:10BF6800F0B5524E336813F0010485B0074640F02F
:10BF78009B804F4B4F4D5049ED1AED082D0445F06D
:10BF880004052846FAF786FD4C4B4D481F60FBF721
:10BF9800C9F9029400F0B1F90446002873D1494A5E
:10BFA80049492846FAF77AFD4648FFF711FB044647
:10BFB800002868D145492846FAF76CFD01F066FF6C
:10BFC800044600285FD102A802F02CF80446002895
:10BFD80059D13F492846FAF75DFD02A9012002F030
:10BFE8002BF8044600284ED13A492846FAF752FD64
:10BFF80002A802F0F1F80446002844D100F044FEFB
:10C00800002843D0344800F033FE336843F002037D
:10C018003360112302A88DF80430FFF7ADFA044607
:10C0280088BB9DF8093002A801338DF80930FFF765
:10C03800A1FA044638BB33689B072CD5264C274900
:10C04800A3692846221DFAF733FDA069211D82B293
:10C0580001A8FFF79FFA0446A8B92148FFF798FA04
:10C06800044680B91F48FFF7CFFE044658B9FFF7CA
:10C0780043FB044638B933681B4943F0010328469B
:10C088003360FAF707FD204605B0F0BD174928468A
:10C09800FAF700FDBDE716492846FAF7FBFC1548F4
:10C0A80002F015FA1349D2E70024ECE77C9100204E
:10C0B8004CE5020064E5020045FE02008091002084
:10C0C800D0E502000060020064FE020084FE020067
:10C0D80099FE0200B0FE0200DC800020E2FE0200B1
:10C0E800960203004691002022FF0200C8FE0200CB
:10C0F80003FF02003DFE020030B51A490B6885B007
:10C1080004460BB1013B0B601748184A6368257851
:10C11800801AC008000440F004008BB90B68144A68
:10C1280014490093012D18BF0A46A3681249FAF76B
:10C13800C9FC63699BB1E06805B0BDE830401847A9
:10C148000A68029222690192A26800920949084A83
:10C15800012D18BF0A460949FAF7CEFCE9E705B0F0
:10C1680030BD00BF889100206CE502004CE502005C
:10C17800BC020300C2020300C8020300EE0203006F
:10C1880008B50C4A0C4B9B1ADB081B0443F004034C
:10C1980050B10A491846FAF77DFC094909480022B6
:10C1A800BDE80840FBF75EBB07491846FAF772FC82
:10C1B8000649F3E74CE502006CE50200940303002E
:10C1C800F4E90200B8570020BA030300C8E90200E6
:10C1D8002DE9F7439846174C174BDFF86C90E41A93
:10C1E800E408D9F8003024040546CDE900230E46BA
:10C1F8000B4617461149024644F00400FAF76EFC54
:10C208002946CDF800803B4632460D48FBF742FBF5
:10C21800054640B9D9F800300133C9F8003028463E
:10C2280003B0BDE8F0830246064944F00200FAF77D
:10C2380035FCF4E76CE502004CE50200E20303007C
:10C24800B857002025040300889100202DE9F34108
:10C25800134B144C144EE41AE40833680093240476
:10C2680005460B460F4690461049024644F0040026
:10C27800FAF728FC294643463A460D48FBF75AFB8D
:10C28800054630B9336801333360284602B0BDE84B
:10C29800F0810246074944F00200FAF7FFFBF4E791
:10C2A8004CE502006CE50200889100202A03030097
:10C2B800B857002067030300014B18700B20704724
:10C2C8008C910020024B002218781A70704700BF2A
:10C2D8008C91002018DF704730B585B005461022D4
:10C2E8000C466846002102F09DF8A40868460195AE
:10C2F8000294FFF7EFFF05B030BD1FB5002304A877
:10C30800CDE901330393022340F8103DFFF7E2FF24
:10C3180005B05DF804FB4FF000534FF480521A60EB
:10C3280000207047084B09480949C01A10B5C008D1
:10C33800000440F00400FAF7ADFB064B06201B682A
:10C34800BDE81040184700BF4CE5020074E5020044
:10C3580058090300989100200A2803D90B38C0B265
:10C36800FFF7AABF7047000070B5054686B00020E9
:10C37800FBF71CFB014690B1244A18212846FAF71E
:10C38800ADFD024648B12248224B23491B1ADB085F
:10C398001B0443F00100FAF781FB06B070BD1822B8
:10C3A800684602F03FF804238DF80030194C184B0A
:10C3B8001A4EE41A1A4B1A6D3368E40824049A4298
:10C3C80044F004041AD117492046FAF763FB164BC8
:10C3D8003168186801F03EFC8DF80100FFF7BCFFDA
:10C3E800D5E901138DF80100684698470F4800F019
:10C3F8002BFB9DF801200E492046CCE701238DF840
:10C4080001306846D5E901139847F2E771C3020085
:10C418004CE5020074E50200D80803009091002062
:10C428009C98002001090300949100202DC302006C
:10C43800300903002DE9F041836888B0044623B928
:10C448009F4940F2CF20FAF75DFE162200210DF138
:10C458000A0001F0E7FF9B4E9B4922788DF80820DF
:10C46800761AF608012336040C2A8DF8093046F0AE
:10C47800040500F2C581934013F4AD7F24D1D9049B
:10C4880007D45B0740F1BC8190492846FAF702FBC4
:10C4980007E028468E49FAF7FDFA8E4B07201B68FD
:10C4A80098479DF809208C492846FAF7F7FAD4E905
:10C4B800011302A898479DF80930012B00F08A81E2
:10C4C800844B05201B6884E1062A844F01D0012A89
:10C4D80001D123693B703B78012B09D0022B75D021
:10C4E8007F4946F00100FAF7D5FA00233B70C8E00F
:10C4F800013A072A64D8DFE802F004631443635B57
:10C50800631E78492846FAF7C5FA724B03201B6860
:10C518009847606901F094F8FFF71EFF8DF809004D
:10C52800BFE771492846FAF7B5FA704BDA6B1B6C0E
:10C5380003920493B5E7236923B9614940F21310C4
:10C54800FAF7E0FDA38A23B95D494FF48A70FAF738
:10C55800D9FD67492846FAF79DFAA18A206901F0B2
:10C5680087F8FFF7F9FE614B8DF80900DA6B1B6C51
:10C578000493E3680392002B93D02069984790E7CF
:10C588005C492846FAF786FA5B495C4801F0EEF800
:10C59800FFF7E2FE01288DF8090082D1002000F0A3
:10C5A80053FA08B9564970E70A238DF8093078E735
:10C5B80054492846FAF76EFA4FF400730593B4E726
:10C5C8003F494FF4BC70FAF79DFD6AE7013A072A24
:10C5D80000F21281DFE812F008001001D200E10039
:10C5E800100101011001600047492846FAF752FA84
:10C5F80001F06EF830B9454946F00100FAF74AFAF9
:10C608000823D2E7626932B9414946F00100FAF7D6
:10C6180041FA0323C9E7C2F30B0343B1334B36494D
:10C628005B6D096813448B4201D03A49EDE7B2F5D6
:10C63800805F06D9384946F00100FAF72BFA04233F
:10C64800B3E72A4F2C497B6D0968D018884206D970
:10C65800009146F001003149FAF734FAD0E77A64DC
:10C66800FA6CBA64254A3B6510683B6300220121D5
:10C678001844FFF7EBFD30B1294946F00100FAF7FD
:10C6880009FA052391E7BB6C00933B6D7A6C254949
:10C698002846FAF717FA04E723492846FAF7FAF979
:10C6A80001F016F80028ABD0104FA18AD7E9143250
:10C6B8009B1A7A6C0B4493423AD91C49A5E700BFF0
:10C6C8007C04030074E502004CE50200DD0403006D
:10C6D8000105030098910020300903000458002048
:10C6E8009908030019050300430503009C980020DE
:10C6F80067050300900503009091002094910020A5
:10C70800BB050300E00503000A0603003106030029
:10C71800660603007F060300A0060300C4060300A4
:10C72800350703004C07030087070300AD07030024
:10C73800374A3B6B1268206903EB020807F148028D
:10C74800FAF7C2FCE368064623B932494FF4F87099
:10C75800FAF7D8FCE368A28A21694046FFF738FD5A
:10C7680008B1E36809E7A38A3A6BBE641A443A63DE
:10C778003A6D049613443B65039392E6264E274987
:10C788002846FAF787F9B36C326D25492846FAF737
:10C798008FF9B36C0493336DEEE728462149FAF715
:10C7A80079F91D48D0E91473426CFB1A934205D0FD
:10C7B8001D4946F00100FAF77BF921E7836CC36451
:10C7C8000021416447652046FFF7CEFD174B1B68E3
:10C7D8000420984708B0BDE8F08115492846FAF7C3
:10C7E80059F90D4B4FF480519A6C1B6D05910091CE
:10C7F800049203930F494BE7064940F29720E2E67B
:10C808000D4946F00300FAF749F90223CDE600BFC7
:10C81800949100207C0403009C980020C407030026
:10C82800E5070300FB070300230803009891002095
:10C83800470803006E080300B9080300836810B5B1
:10C848008BB10A4A1821FAF749FB044648B108484F
:10C85800084B0949C01AC008000440F00200FAF762
:10C8680019F9204610BD0724FBE700BF3DC40200AC
:10C8780074E502004CE502006004030038B5054683
:10C88800C0B10120FFF77CFC044648B900F0C6FEA1
:10C8980000F01EFF30B9084B00201D60FFF70CFDAB
:10C8A800204638BD0549064800F060FF0128F2D04F
:10C8B8000324F5E70724F3E79891002090910020DE
:10C8C8009491002010B50022044658210430FAF74C
:10C8D800FBFB23681B1A5842584110BD2DE9F0474D
:10C8E80016464FF460721F46054688461E4C01F0F6
:10C8F8003AFD1E4BE41AE408240444F0040A814675
:10C9080050B91B495046FAF7C5F816B90020BDE8DA
:10C91800F0874846B047F9E716495046FAF7BAF89B
:10C928002A4615495046FAF7B9F800220121284647
:10C93800FFF78CFC30B1114944F00100FAF7AAF86E
:10C948000320E4E74FF460724146384601F041FDA8
:10C9580033464FF4607239462846FFF739FC002801
:10C96800D4D00749E8E700BF7CE502004CE50200A7
:10C97800150C03005F0C0300730C0300930C0300F9
:10C98800B60C030070B50C4C054600225821201D3A
:10C99800FAF79AFB00222060C32104F51870FAF711
:10C9A80093FB2A46C4F85C022146044B0448BDE8C0
:10C9B8007040FFF793BF00BF9C9800209C91002017
:10C9C80000F00700F8B5164B164C174DE41AE408AA
:10C9D8000E46240407462A68144944F00300FAF76F
:10C9E8005DF83368013313D1114940F27910FAF731
:10C9F80089FB3A460F4B28683146FFF76FFF02461E
:10CA080060B144F001000C49BDE8F840FAF746B8B7
:10CA18003046FFF757FF0028EBD1E5E7F8BD00BF28
:10CA28004CE502007CE5020008580020500B03008A
:10CA38007A0B03001C950020D80B03000149FFF76F
:10CA4800C1BF00BF00F0070038B505460020FFF75A
:10CA580099FF044618B903492846FFF7B3FF204653
:10CA680038BD00BF9C9800202DE9F8435F4B604C0F
:10CA78006049E41AE408240444F0040905464846D9
:10CA8800FAF708F82846FFF77BFB024638B15A49FF
:10CA980044F00100FAF702F80320BDE8F88357488C
:10CAA800036801333DD0FFF70DFF0546544B554F42
:10CAB8001E683268013298467BD03046FFF702FF85
:10CAC80000287AD07368012B00F08280002206F5D6
:10CAD8001870C321FAF7F8FAD6F85C321A1A5642D7
:10CAE800564105B348494846F9F7D4FF4FF46072F8
:10CAF8004249444801F06DFC7EB344494846F9F781
:10CB0800C9FFD8F8001042485422043101F061FCF2
:10CB1800D8F800103F484FF432725C3101F059FCEC
:10CB28001BE01546C2E783420AD13B4944F00300A3
:10CB3800F9F7B0FF4FF46072D8F800103148EDE70C
:10CB4800364944F00200F9F7A5FF4FF4607200215E
:10CB58002C4801F067FC02237B607D68012D1FD102
:10CB68002F4944F00300F9F795FF2E49402201F5BB
:10CB7800E47001F02EFC2C491C2201F5E47001F050
:10CB880028FC2A4987F8A1520023042201F28620B2
:10CB980087F8603287F8E23201F01BFC02237B60E1
:10CBA8000020FFF751FF00283FF477AF02462049E5
:10CBB8006EE7002DC4D0002694E7002DC0D012499E
:10CBC8004846F9F767FF4FF460720C493846A5E705
:10CBD800002DAAD048460C49F9F75CFF4FF4607263
:10CBE8000649384601F0F5FB87E700BF4CE502002F
:10CBF8007CE50200A0090300C309030000F0070058
:10CC0800085800209C980020EE090300030A03003E
:10CC1800A0980020F89800202D0A0300860A030037
:10CC2800EA0A0300F8990020389A0020B8980020F2
:10CC3800160B030029DF704738B50C4D0446D5F8AC
:10CC4800643378B101330FD1002218210430FAF788
:10CC58003BFA21462060072205F55970BDE83840A7
:10CC6800FFF7E8BF0E2038BD0820FCE700F00700FA
:10CC780008B528B11C22034901F0ABFB002008BD10
:10CC88000E20FCE764F3070010B5064C00221821BB
:10CC98002046FAF719FA54F8043C1B1A584258412E
:10CCA80010BD00BF68F3070008B50F4BD3F8242365
:10CCB800013203D1D3F86433013313D00B4B0C4842
:10CCC8000C49C01AC008000440F00400F9F7E2FE5D
:10CCD8004FF4FE20FBF756FBC92203494FF4FE2010
:10CCE800FBF768FB002008BD9C9800204CE502007B
:10CCF80084E50200EE0C03002DE9F843144B154CB3
:10CD0800DFF86090144D1549E41AE408A5EB09050D
:10CD18002404ED0844F0040407462A462046F9F79F
:10CD2800BDFE0026AE4202D14FF000080BE059F8D4
:10CD3800363038469847804640B10346324608495F
:10CD48002046F9F7B5FE4046BDE8F8830136E9E725
:10CD58004CE502004CE5020040E502007A0D0300B4
:10CD68009E0D030038E502002DE9F843154B164CDB
:10CD7800DFF86490154D1649E41AE408A5EB090597
:10CD88002404ED0844F0040407462A462046F9F72F
:10CD980085FE0026AE4202D14FF000080CE009EBF8
:10CDA800C60338465B689847804640B1034632461A
:10CDB80008492046F9F77CFE4046BDE8F88301366D
:10CDC800E8E700BF4CE502004CE5020040E5020040
:10CDD8002B0D0300500D030038E5020008B50C22A6
:10CDE800002101F01FFB024B00221A6308BD00BF9F
:10CDF8009C98002043F204031A68084B9A4201BF2A
:10CE080043F20803186800F6FF7020F47F600CBF37
:10CE180020F00F004FF48050704700BFDBE5B151A0
:10CE280008B5FFF7E7FF054B9B69184400F6FF704C
:10CE380020F47F6020F00F0008BD00BF9C98002000
:10CE48004FF48050704700002DE9F04F89B08046BC
:10CE580001920593674A684B04919B1ADB081B04EF
:10CE680043F00404654902932046F9F713FE42464D
:10CE78006349644E644D654F2046F9F70FFE049BE5
:10CE88006349002B0CBF32462A462046F9F706FEB6
:10CE9800019B6049002B0CBF32462A462046F9F711
:10CEA800FDFD059B5C49002B0CBF32462A462046F7
:10CEB800F9F7F4FD43F2040358491A68584B204621
:10CEC8009A4214BF32462A46F9F7E8FD55492046EA
:10CED800F9F7E0FDBB693A6A53492046F9F7E8FDDE
:10CEE8007B6AFA6A51492046F9F7E2FD4FF00009DA
:10CEF8000697B346AA465FFA89F6012E50D0022E4D
:10CF08005DD0FFF78DFF019A0346002A46D0069AA6
:10CF1800156A6A1E55425541454F9F4205D24549FB
:10CF28000393B120FAF7EEF8039B0793FF1A049BCB
:10CF38004149474538BF01234A4620460393F9F73C
:10CF4800ADFD079B3D491A462046F9F7A7FD474521
:10CF58002CBF5A4652463A492046F9F79FFD002D04
:10CF68000CBF5A46524637492046F9F797FD039BAE
:10CF78003549002B0CBF5A4652462046F9F78EFD1C
:10CF8800039B03B3FDB9B9F1020F04D009F10109FC
:10CF9800B9F1030FAFD1474517D321E0019DBBE796
:10CFA800FFF728FF059A03463AB943F204021568C9
:10CFB8001B4AAD1A18BF0125AEE73546ACE7012577
:10CFC8004FF48053A8E7474509D2029B1F4943F015
:10CFD8000200F9F75FFD042009B0BDE8F08F36B113
:10CFE80020461B49F9F756FD1A48FFF7F7FE0020BF
:10CFF800F2E700BF4CE502004CE50200CA0D030051
:10D00800E80D0300020E0300FD0D03009C980020AC
:10D01800080E0300190E0300270E03003C0E030040
:10D02800DBE5B1514C0E03005B0E03007B0E0300E1
:10D03800003002009B0E0300F60E0300000F0300F1
:10D04800150F03002A0F03003D0F03004E0F0300C6
:10D058007A0F0300B498002010B5084C4FF4007202
:10D06800FF21204601F0DEF920220021A4F124004E
:10D0780001F0D8F9002344F82C3C10BDF8980020A2
:10D088002DE9F04F4049414E8A6B414DDFF8289118
:10D09800DFF828A1DFF828B185B06F465C31384643
:10D0A800FBF75EFB97E80F004FF0000886E80F00DB
:10D0B800384BF3604FF447724146284689F80080A0
:10D0C800CAF80080CBF8008001F0ACF92A46324952
:10D0D8003046FBF7E4FD044650B93048304B31493F
:10D0E800C01AC008000440F00100F9F7D3FC14E0AE
:10D0F80099F80090B9F1000F04D095F86C312C78AC
:10D10800A3B374B1264B25482749C01AC0080004A8
:10D1180040F00100F9F7BEFC0024204605B0BDE848
:10D12800F08F95F87241002CF7D0DBF80020DAF880
:10D1380000103846FBF714FB97E80F0086E80F004D
:10D148004FF4B272414605F5BA7001F06BF905F576
:10D15800BA7216493046FBF7A2FD044680B90F485B
:10D168000F4B1349C01AC0080004BCE7002CD4D0E8
:10D17800AC79002CD1D008350E4B4C461D60CCE75D
:10D1880005F5BA75F8E700BF9C980020689F002055
:10D198004C9C002059D20200A8FC02008CE5020039
:10D1A8004CE5020095140300C2140300F4FB0200CE
:10D1B800E114030024A00020489C0020449C002087
:10D1C800409C002090F8553013F0FB0F10B508D1A3
:10D1D80090F864202AB1846E74B30C600124204650
:10D1E80010BD13F0010403D090F8564004B1846DCB
:10D1F8009B07F1D590F85C30002BEDD00F4B026EF9
:10D20800C3F5FC239A4201D81444E5E70C490D48BC
:10D21800401AC00800040C4940F00100F9F748FC26
:10D228000424074B07480949C01AC008000440F005
:10D238000100F9F72FFCD2E70F24F2E700600200A3
:10D248004CE502008CE50200301503004D15030083
:10D258005B68DA68134B9A4230B408D1124C2268E2
:10D2680012B912490A6822B1114B00221A7030BC57
:10D278007047D0E90132981813F9015B002DA0EB33
:10D288000302F9DB23600A4B0A600121197009487F
:10D29800094B0A49C01AC008000440F0040030BC19
:10D2A800F9F7FCBBF4FB0200449C0020409C0020E2
:10D2B800489C00208CE502004CE50200D0120300D7
:10D2C80000B591B0FBF72CFF18B10D49DB20F9F739
:10D2D80019FF20220B496846FBF772FF40236A4674
:10D2E80009490A48FBF774FE18B10549E520F9F722
:10D2F80009FF074B01221A7011B05DF804FB00BF4B
:10D30800DE0F0300BCF10200789F0020C4F0020089
:10D318001C9C00202DE9F043A3B081460F46164619
:10D32800984678222023002104A8029301F07AF875
:10D3380000230393404B1B780BB9FFF7C1FF3F4C09
:10D348003F4B4049E41AE408240444F00305284606
:10D35800F9F7A0FB47B944F002003B49F9F79AFBFB
:10D36800132023B0BDE8F083B9F1000F05D028469B
:10D378003649F9F78FFB1620F3E72A9A3449DFF884
:10D38800F8902846F9F78AFB02AB0193CDF8009094
:10D398002A9B3049424604A8FBF7A8FE002849D139
:10D3A800402E47D1DFF8D48032463946404601F056
:10D3B80010F829492846F9F76DFB20214046FBF76C
:10D3C8000CFF4A46CDE90086029B244903A8FBF7D7
:10D3D8001BFE024640B344F00100214944F0040416
:10D3E800F9F75CFB1F492046F9F754FB32464146E2
:10D3F8002046F9F791FB1C492046F9F74BFBBDF88D
:10D40800082049462046F9F787FB18492046F9F7CE
:10D4180041FB324616492046F9F77EFBF9F7ACF98D
:10D428000028FBD105209CE728461249F9F732FB72
:10D43800012096E70A2094E71C9C00208CE5020056
:10D448004CE50200031203002B1203003F120300F5
:10D45800561203004CFB020071120300789F002053
:10D4680082120300A4120300AF120300B5120300D6
:10D47800BCF10200C1120300C09F0020E09F002001
:10D4880043F2040313B51A68224B9A423FD042F282
:10D4980004014458E11A4C424C419A4234D142F2B8
:10D4A8000403C35893422FD14FF440531B78142BD5
:10D4B80081BF43F21403184A1B68B3FBF2F300F56B
:10D4C800005298BF00231278142A82BF42F2140235
:10D4D80011498258114888BFB2FBF1F21049A0EBFC
:10D4E800010098BF00220F490092C00893424FEAFA
:10D4F80000400D4A40F0030018BF0A460B4914BF0C
:10D5080001240024F9F7DEFA204602B010BD0024F9
:10D51800C3E700BFDBE5B15140420F008CE50200D4
:10D528004CE502003E100300441003004A100300BB
:10D538002DE9F043ABB006460F4690461C467822CC
:10D54800202300210CA8039300F06CFF294B1B78C3
:10D558000BB9FFF7B5FE2CB13146202204A8FBF722
:10D5680013FE04AE244B254C2549DFF8AC90E41A91
:10D57800E408240444F0040543463A462846F9F7EB
:10D5880097FA03AB01933A46CDF8009043461D49FC
:10D598000CA8FBF7ABFD024640B144F001001A4964
:10D5A800F9F77CFA00202BB0BDE8F0832022314641
:10D5B800484600F0D8FED8B1144944F00200F9F703
:10D5C80069FA13492846F9F765FA202231462846B0
:10D5D800F9F7A2FA0F492846F9F75CFA20224946DA
:10D5E8002846F9F799FAF9F7C7F80028FBD1DAE7DE
:10D5F8000120D8E71C9C00204CE502008CE50200C5
:10D60800AD1003004CFB0200E010030011110300F1
:10D618002B1103003D1103001D9C0020064B9B6B42
:10D6280010B5064C2BB1FFF72BFD10B10123237069
:10D6380010BD0023FBE700BF9C98002020A000201D
:10D6480010B5044658B1B0F5007F0AD8064B002241
:10D658001A70FFF701FD054B01209C6310BD0320E4
:10D66800FCE70420FAE700BF20A000209C980020D7
:10D6780070B5134C0646E06BA36B42189A420D46F0
:10D688000BD9104B10481149C01AC008000440F0CB
:10D698000100F9F7FFF9032070BD5C300A46204409
:10D6A800314600F096FEE36B04F140022B44294614
:10D6B8003046E363F9F708FD20640120ECE700BF7A
:10D6C8009C9800204CE502008CE502004D110300F7
:10D6D800014B1878704700BF20A00020F7B51C4CFC
:10D6E80094F86C217AB394F8D802B4F8DA2204F5E5
:10D6F800377104F5B874174E174D336800932B68CB
:10D70800FFF708FE0128074605D1201D00F0A6FAFC
:10D718000128074614D0114B114C1249E41AE408A9
:10D72800240444F0020044F00404F9F7B3F90E4964
:10D738002046F9F7AFF9328829682046F9F7ECF95D
:10D74800384603B0F0BD114610460434D3E700BF95
:10D758004C9C0020409C0020449C00204CE502008A
:10D768008CE50200DF110300F5110300334BD3E908
:10D778000E329A422DE9F04106460D460DD0304B47
:10D7880030483149C01AC008000440F00100F9F7D8
:10D7980081F908242046BDE8F0812C4F97F80080D5
:10D7A800B8F1000F09D0FFF73BFB294B3060294641
:10D7B8001868BDE8F041FFF705BDFFF761FC80B3CD
:10D7C800FFF78CFF0128C6F800800446C5F80080E2
:10D7D80019D11F4B29461868FFF7F4FC01280446A5
:10D7E80011D1034642462868164D4146FFF72CFBE7
:10D7F800134BED1AED082D0440B1164945F0010010
:10D80800F9F748F90424FFF727FCC3E7FFF708FBFB
:10D8180011493060024645F00400F9F73FF93C70C1
:10D82800B8E7074B07480D49C01AC008000440F084
:10D838000100F9F72FF90524ACE700BF9C980020F8
:10D848004CE502008CE502007011030020A00020C6
:10D8580024A000208B110300A6110300C2110300AD
:10D8680070B50D461646044620B907494FF42E7088
:10D87800F9F748FC3246294604F172000123BDE855
:10D888007040FFF755BE00BFDE0F0300037837B5C1
:10D898000C461146032B2DD8DFE803F0150217209C
:10D8A800D0F8015000222046F9F70EFC85420AD034
:10D8B8001448154B1549C01AC0080004012240F04D
:10D8C8000400F9F7EBF8012012E00A46002321468C
:10D8D800013003B0BDE83040FFF72ABE009123466F
:10D8E800411C40220020FFF715FD431E58425841B5
:10D8F80003B030BD4FF477700549F9F703FC0020F9
:10D90800F6E700BF8CE502004CE502008A10030030
:10D91800DE0F03002DE9F041A2B004460E4617467B
:10D9280000217822984604A8202303939DF8A0504C
:10D9380000F078FD41220021204600F073FDB6F882
:10D9480094300BB196F896502570032D35D8DFE842
:10D9580005F009020F2C002241463846F9F7B4FBBE
:10D96800C4F80100424639462046FFF78FFF19E008
:10D9780003AB0193631C00933A464346144904A839
:10D98800FBF7B4FB0028EDD0FAF76EFB114A124BF7
:10D9980012499B1ADB081B04024643F00100F9F701
:10D9A8007DF8002022B0BDE8F081B6F8982006F195
:10D9B8009A01601C00F00DFDD4E70748054B0849A3
:10D9C800C01AC00800042A4640F00100E7E700BF7B
:10D9D8004CFB02004CE502008CE502008C0F0300B2
:10D9E800BD0F03002DE9F0478A4B1C68A4B005461B
:10D9F800884691460A4601462046FFF731FF00282F
:10DA080000F0068194F85560002E3AD14FF0010AD3
:10DA1800CDF800A043462A46214613A8FFF77AFF0F
:10DA280038B90524B9F1000F40F0D380FFF714FB93
:10DA380048E0B9F1000F42D0412213A97648774F48
:10DA480000F0C7FC764B77487749C7F82CA0C01A76
:10DA5800C008000440F00400F9F71CF894F892306C
:10DA68003E6213B194F893300BB96368BB6000222F
:10DA780041462846F9F728FB684B0124C3E9098089
:10DA8800AAE04122002102A800F0CCFC06F0010A1D
:10DA98004122002113A806F0020600F0C3FCBAF1E7
:10DAA800000F40F09E80002E40F08C805F494FF4BC
:10DAB8005970F9F727FBB9F1000F40F08680574BF2
:10DAC80001245C61204624B0BDE8F087A36D03F50E
:10DAD800FF5203F6FF731F32C3F30B03D31A42F24C
:10DAE8000802AA589A4206D24E484D4B5049C01ACD
:10DAF800C008000487E02846FFF7C2FC70B1494F10
:10DB0800474B4C49FF1AFF083F0447F00200F8F75B
:10DB1800C1FF1EB9484947F0010076E00123009390
:10DB2800A36D2A46214602A8FFF7F4FE00283FF419
:10DB380078AFCEB1A36DEA18A8EB030300210091DA
:10DB480013A82146FFF7E6FE00283FF46AAF9DF8C8
:10DB58004C304BB13348324B3849C01AC008000426
:10DB680040F00200F8F796FFB9F1000FA7D0BAF11C
:10DB7800000F2AD02846FFF783FC10B13048FFF782
:10DB88002DF9412202A92F4800F023FC002E234B37
:10DB980014BFAC22A522DA62A26D5A63002E3FF4AC
:10DBA80066AF412213A9284800F013FC94F892307C
:10DBB80023B194F89330002B7FF459AF174B626868
:10DBC800DA6054E743462A46B8E7144BAA22DA62D9
:10DBD800E4E71E48FFF702F9FFF73EFA0F4B9D6492
:10DBE80070E742F20403EA5803F1A34303F547132D
:10DBF80003F2D7539A423FF469AF0A48084B1449D5
:10DC0800C01AC008000440F00100F8F743FF08E715
:10DC1800172407E724A000203D9B00209C980020A3
:10DC28004CE502008CE50200ED120300DE0F030054
:10DC380066130300CF1303001014030051140300EC
:10DC4800B4980020FC9A00207E9B0020C0980020F9
:10DC5800151303000122FFF7C5BE0000F8B50446FE
:10DC680018B94F49C420F9F74DFA94F854309BB1CC
:10DC780094F8550003280FD894F86E30032B17D06A
:10DC8800484B49484949C01AC008000440F00100FF
:10DC9800F8F700FF1420F8BD4348424B4449C01A26
:10DCA800C008000440F00100F8F7F4FE0F20F2E786
:10DCB80094F892301BB194F89330002B65D1237AF5
:10DCC80033B93948374B3B49C01AC0080004E9E763
:10DCD800E368342B0BD0334B33483749C01AC0089C
:10DCE800000440F00200F8F7D5FE1120D3E743F214
:10DCF8000402238A1168314A91423DD153B16269C5
:10DD0800DAB104F11405DBB2002243F20C06D1B2F9
:10DD18008B420BD8234B24482949C01AC008000459
:10DD280040F00200F8F7B6FE1220B4E7318855F843
:10DD380022708F4204D00132E9E7B0B9012BE9D84B
:10DD4800237823B3012863681E4A1BD8926893423C
:10DD58001BD2144B14481C49C01AC008000440F0D8
:10DD68000200F8F797FE102095E710F1FF3318BF6F
:10DD78000123002BE4D1CDE713B16369002BC9D18E
:10DD88002378F6E7D2689342E3D9012083E7012894
:10DD980081D00548034B0D49C01AC008000481E72B
:10DDA8007E1503004CE5020094E50200F915030016
:10DDB800E21503000C1603001B160300DBE5B15146
:10DDC8002E1603009C9800203E16030052160300EE
:10DDD80010DF704711DF704713B5044609496846DC
:10DDE800FAF7EEF8019808B902B010BDD0E9003191
:10DDF8002046984718B16846FAF7FCF8F2E7112070
:10DE0800F2E700BF8416030013B5044607496846C5
:10DE1800FAF7D6F8019B0BB902B010BD2046D3E93A
:10DE2800002190476846FAF7E5F8F3E79C160300E7
:10DE3800064B9A6822B11A6822F480021A60704769
:10DE4800034B4FF48002C3F880207047046A002017
:10DE580000E100E00B4991F816335A09EC2313410D
:10DE6800DB0706D5084B9A683AB94FF480030B6074
:10DE7800704742F20200FBF71BBA1A6842F48002AC
:10DE88001A60704700E100E0046A0020F7B5184FF7
:10DE98003C785CBB174E012520463570FFF79CFF88
:10DEA800112820D02046FFF7AFFF134B18680190C8
:10DEB80002A800F8054DF9F7B7F8104901A8FFF7CF
:10DEC80087FF0446B0FA80F0400938709DF80300D7
:10DED800F9F7DAF83CB90A4B34701C70FFF7BAFF4F
:10DEE8002846FFF791FF204603B0F0BD0824FAE763
:10DEF80029A0002028A000207D1603008D92020092
:10DF08002AA00020F7B5154F3B7813B3144E012013
:10DF18003070FFF761FF11284FF000051BD0022079
:10DF2800FFF772FF02A800F8015DF9F77DF8FFF727
:10DF380051FF04469DF807003D70F9F7A5F82CB984
:10DF48003470FFF775FF0320FFF75EFF204603B02C
:10DF5800F0BD0824FAE72C46F8E700BF29A0002006
:10DF680028A00020054B1B7833B1054B1B780BB15B
:10DF7800FFF7C8BFFFF78ABF0820704728A0002016
:10DF880029A00020014B1878704700BF29A0002065
:10DF980007B508496846FAF713F8019B13B903B0A7
:10DFA8005DF804FBD3E9002090476846FAF722F8A9
:10DFB800F3E700BF90160300FFF7EABF60DF704782
:10DFC80069DF704761DF704730B5114DADF5017DF0
:10DFD8004FF4FA740DF1020103A8ADF80240FFF7FF
:10DFE800F1FF70B9294601A8F9F7EAFF029B002B57
:10DFF800F0D003A8D3E90021904701A8F9F7FAFF68
:10E00800F4E7052801D0FBF753F90DF5017D30BD84
:10E0180020190300024B1B780BB1FFF7D5BF7047DF
:10E028002BA0002018B1034B0360002070470E207E
:10E03800704700BFB857002030B5054685B00C467C
:10E04800002900F0B5805B4B0B600C22002101A871
:10E0580000F0E8F901238DF8063022688DF80450A5
:10E06800062301A92020ADF80830FFF7A9FF60B109
:10E07800F9F7FAFF504A514B51499B1ADB081B0428
:10E08800024643F00100F8F709FD0C22002101A81F
:10E0980000F0C8F901238DF805302268002301A992
:10E0A80040208DF806308DF80730FFF789FF60B102
:10E0B800F9F7DAFF404A414B42499B1ADB081B0437
:10E0C800024643F00100F8F7E9FC0C22002101A800
:10E0D80000F0A8F9F72322688DF8045001A923203D
:10E0E800ADF80630FFF76CFF60B1F9F7BDFF324AB3
:10E0F800324B35499B1ADB081B04024643F00100EA
:10E10800F8F7CCFC0C22002101A800F08BF90120C3
:10E1180022688DF8040001A9FFF752FF60B1F9F7F2
:10E12800A3FF254A254B29499B1ADB081B040246F5
:10E1380043F00100F8F7B2FC0C22002101A800F01E
:10E1480071F94FF4B0632268019301A9A120FFF788
:10E1580037FF60B1F9F788FF174A184B1C499B1A1B
:10E16800DB081B04024643F00100F8F797FC0C2279
:10E17800002101A800F056F99DF8043022686FF3D9
:10E18800000301A9A0208DF80430FFF719FF68B13A
:10E19800F9F76AFF084A094B0E499B1ADB081B046A
:10E1A800024643F00100F8F779FC002005B030BDC5
:10E1B8000E20FBE7B85700204CE50200ACE5020052
:10E1C800B0160300F6160300421703008917030070
:10E1D800D517030026180300F8B506460768FFF7A9
:10E1E800EDFE3368BB4205461DD9194B194C1A4937
:10E1F800E41AE408240444F002042046F8F74AFC30
:10E20800336816493A462046F8F752FC4FF08053D7
:10E218003268D3F80C3112499B0203F100539A1A61
:10E228002046F8F73BFC25B90E4B01221A70284608
:10E23800F8BD2846F9F718FF054A064B0A499B1A04
:10E24800DB081B04024643F00100F8F727FCEEE761
:10E258004CE50200ACE5020079180300A818030099
:10E26800D91803002BA00020031903004BDF7047C7
:10E278001FB50D4C01A8FFF7F9FF70B9214602A898
:10E28800F9F79EFE039B002BF4D00198D3E90021F7
:10E29800904702A8F9F7AEFEF4E7052801D0FBF78E
:10E2A80007F804B010BD00BF381903007F2805D84F
:10E2B800034B185C034B5B5C1840704700207047A9
:10E2C80050190300D0190300A0F16103192B98BF5E
:10E2D80020387047A0F14103192B98BF20307047B0
:10E2E8007F2805D8034B185C034B5B5C18407047CC
:10E2F8000020704750190300D0190300A0F16103F2
:10E30800192B98BF20387047A0F14103192B98BFEB
:10E31800203070477F299ABF017001206FF02E00CE
:10E3280070475AB10A787F2A0AD800B102600021E2
:10E3380019605960501A18BF0120704700207047B3
:10E348006FF02E007047000008B5034B5B689B68B0
:10E358001B68984708BD00BF0C58002008B5092164
:10E36800FFF7F2FF08BD92B370B4134640EA01020A
:10E3780012F0030F17D05A1E10D004780B789C4265
:10E388000CD1431C4C1C024418462146934205D02C
:10E398000133013406780D78AE42F5D000780B7859
:10E3A800C01A70BC70470F2BE5D904680A689442FC
:10E3B800E1D1041D0A1D20461146043B042BDAD97D
:10E3C8000434043206680D68AE42F4D0D3E7002066
:10E3D8007047844640EA010313F0030F18D18446BE
:10E3E800202A0BD32DE9F007B1E8F807A0E8F807D1
:10E3F800A2F12002202AF7D2BDE8F007042A07D3A9
:10E4080051F8043B40F8043BA2F10402042AF7D275
:10E41800002A05D011F8013B00F8013B013AF9D177
:10E42800604670478446002A2DD010F0030F04D0B0
:10E4380000F8011B013A26D0F7E7C9B241EA0121E9
:10E4480041EA0141202A12D3A2F120022DE9F0036A
:10E458000B460C460D460E460F4688468946A0E8F0
:10E46800FA03203AFBD2BDE8F00320320BD0042A8D
:10E4780005D340F8041B043A05D0042AF9D200F861
:10E48800011B013AFBD160467047024610F0030FAA
:10E4980016D111F0030F13D12DE9F0004FF0013719
:10E4A8004FF0803351F8044BA4EB070525EA040527
:10E4B8001D4002D142F8044BF4E7A1F10401F0BC7D
:10E4C80011F8013B02F8013B002BF9D1704700F12C
:10E4D800010110F0030F11D010F8012B002A23D0EE
:10E4E80010F0030F0AD010F8012B002A1CD010F0EE
:10E4F800030F03D010F8012B002A15D02DE9700066
:10E508004FF001324FF0803350F8044BA4EB020572
:10E5180025EA04051D4000D1F6E7A0F1040070BC0F
:0EE5280010F8012B002AFBD1A0EB0100704778
:08E5380069BF020055B60200A4
:0CE540000000000003000000A18E02009B
:10E54C0039E70200000004045EE80200000000004D
:10E55C0029FB020000000404B002030000000404C4
:10E56C0052040300000004048C090300000004049E
:10E57C00DD0C030000000404150D0300000004046E
:10E58C001D150300000004046616030000000404BB
:10E59C00AEE9020000000404A81603000000030307
:10E5AC002C190300000003034419030000000303AB
:10E5BC00645800202C590020345900206C5800203D
:10E5CC0018000000F88000203491002045910020B4
:08E5DC0000810020F4000000A2
:10E5E40048E6020000000000B3E60200CC57002019
:08E5F400BDB7020000000000A9
:08E5FC00697B02000000000031
:08E60400297D02000000000066
:10E60C001DE002000000000079E2020000000000A2
:08E61C00857C020000000000F3
:10E62400000000000000000001C102000010000012
:04E6340000000800DA
:10E6380000000000000000000338FDD8704700000B
:10E64800DD63020049640200D9630200433A5C6E4C
:10E658006F726469635F73656D695C6E5246355F9E
:10E6680053444B5F31352E332E305F353961633378
:10E6780034355C636F6D706F6E656E74735C6C6956
:10E68800627261726965735C6C6F675C7372635CFC
:10E698006E72665F6C6F675F64656661756C745FE8
:10E6A8006261636B656E64732E63007274745F6C71
:10E6B8006F675F6261636B656E6400433A5C6E6F9F
:10E6C800726469635F73656D695C6E5246355F534A
:10E6D800444B5F31352E332E305F35396163333427
:10E6E800355C636F6D706F6E656E74735C6C6962B8
:10E6F8007261726965735C6C6F675C7372635C6E80
:10E7080072665F6C6F675F66726F6E74656E642E9B
:10E7180063000000586900207F000000D8690020CD
:10E728004261636B656E647320666C7573686564BB
:10E73800006170700000000073E70200B8E7020093
:10E7480078E70200C0E70200C8E70200D0E702004D
:10E75800D8E70200E0E70200E8E7020020253032AF
:10E768007800202020007C002563001B5B306D00B2
:10E778001B5B313B33316D0025734C6F677320642D
:10E78800726F70706564202825642925730D0A004E
:10E798003C25733E2025733A20000000000000004D
:10E7A800F0E70200F6E70200FEE7020003E80200D5
:10E7B8001B5B313B33306D001B5B313B33326D00EB
:10E7C8001B5B313B33336D001B5B313B33346D00D6
:10E7D8001B5B313B33356D001B5B313B33366D00C2
:10E7E8001B5B313B33376D006572726F7200776166
:10E7F800726E696E6700696E666F00646562756740
:10E8080000433A5C6E6F726469635F73656D695C3F
:10E818006E5246355F53444B5F31352E332E305F91
:10E82800353961633334355C636F6D706F6E656E57
:10E8380074735C6C69627261726965735C75746922
:10E848006C5C6170705F7574696C5F706C61746624
:10E858006F726D2E63006D656D5F6D6E677200433C
:10E868003A5C6E6F726469635F73656D695C6E5262
:10E8780046355F53444B5F31352E332E305F353983
:10E8880061633334355C636F6D706F6E656E74737E
:10E898005C6C69627261726965735C62616C6C6FF1
:10E8A800635C6E72665F62616C6C6F632E630043BB
:10E8B8003A5C6E6F726469635F73656D695C6E5212
:10E8C80046355F53444B5F31352E332E305F353933
:10E8D80061633334355C65787465726E616C5C664F
:10E8E8007072696E74665C6E72665F667072696E6D
:10E8F80074662E6300303132333435363738394157
:10E908004243444546433A5C6E6F726469635F7381
:10E91800656D695C6E5246355F53444B5F31352EE9
:10E92800332E305F353961633334355C657874650F
:10E93800726E616C5C667072696E74665C6E72662B
:10E948005F667072696E74665F666F726D61742E51
:10E958006300433A5C6E6F726469635F73656D69E7
:10E968005C6E5246355F53444B5F31352E332E3043
:10E978005F353961633334355C636F6D706F6E6515
:10E988006E74735C6C69627261726965735C6673DC
:10E99800746F726167655C6E72665F6673746F72BE
:10E9A8006167652E63006E72665F6673746F72616D
:10E9B800676500000010000004000000010000006E
:10E9C800017A0200257A0200357A0200A17A020053
:10E9D800457A02000D7A0200117A0200157A0200C7
:10E9E800001000000400000001000000AD7B0200E0
:10E9F8008D7B02007D7B0200B57D0200697D0200EF
:10EA0800517B0200557B0200597B0200433A5C6E41
:10EA18006F726469635F73656D695C6E5246355FDA
:10EA280053444B5F31352E332E305F3539616333B4
:10EA380034355C636F6D706F6E656E74735C6C6992
:10EA4800627261726965735C6D656D6F626A5C6E36
:10EA580072665F6D656D6F626A2E6300433A5C6E25
:10EA68006F726469635F73656D695C6E5246355F8A
:10EA780053444B5F31352E332E305F353961633364
:10EA880034355C636F6D706F6E656E74735C6C6942
:10EA9800627261726965735C6578706572696D65CB
:10EAA8006E74616C5F73656374696F6E5F766172B3
:10EAB800735C6E72665F73656374696F6E5F6974A9
:10EAC80065722E6300556E6B6E6F776E206572727D
:10EAD8006F7220636F6465000000000008EC02009C
:10EAE8000100000014EC02000200000032EC0200F9
:10EAF8000300000053EC02000400000066EC020072
:10EB08000500000077EC0200060000008BEC020014
:10EB180007000000A3EC020008000000BBEC0200A4
:10EB280009000000D3EC02000A000000ECEC02002F
:10EB38000B00000004ED02000C0000001BED0200B9
:10EB48000D0000002FED02000E00000041ED020054
:10EB58000F00000050ED02001000000064ED0200FC
:10EB6800110000007BED0200120000008AED020097
:10EB7800130000009FED020080000000B3ED0200CA
:10EB880081000000D4ED020082000000F0ED0200D8
:10EB9800830000000CEE0200840000002AEE020050
:10EBA800850000004BEE02008600000070EE0200B7
:10EBB8009000000087EE020091000000A5EE020020
:10EBC80092000000C3EE020000820000D8EE0200AE
:10EBD80001820000F6EE02000282000012EF02003D
:10EBE800008400002EEF02000184000052EF0200B2
:10EBF800028400007CEF020003840000A1EF020001
:10EC08004E52465F53554343455353004E52465F59
:10EC18004552524F525F5356435F48414E444C450C
:10EC2800525F4D495353494E47004E52465F455235
:10EC3800524F525F534F46544445564943455F4EE1
:10EC48004F545F454E41424C4544004E52465F4545
:10EC580052524F525F494E5445524E414C004E520B
:10EC6800465F4552524F525F4E4F5F4D454D004EE5
:10EC780052465F4552524F525F4E4F545F464F5572
:10EC88004E44004E52465F4552524F525F4E4F54CB
:10EC98005F535550504F52544544004E52465F45BD
:10ECA80052524F525F494E56414C49445F5041526F
:10ECB800414D004E52465F4552524F525F494E56A3
:10ECC800414C49445F5354415445004E52465F45B8
:10ECD80052524F525F494E56414C49445F4C454E43
:10ECE800475448004E52465F4552524F525F494E74
:10ECF80056414C49445F464C414753004E52465F8B
:10ED08004552524F525F494E56414C49445F444127
:10ED18005441004E52465F4552524F525F4441544F
:10ED2800415F53495A45004E52465F4552524F5231
:10ED38005F54494D454F5554004E52465F45525217
:10ED48004F525F4E554C4C004E52465F4552524F03
:10ED5800525F464F5242494444454E004E52465F28
:10ED68004552524F525F494E56414C49445F4144C7
:10ED78004452004E52465F4552524F525F425553DD
:10ED880059004E52465F4552524F525F434F4E4EC6
:10ED98005F434F554E54004E52465F4552524F52B4
:10EDA8005F5245534F5552434553004E52465F45B7
:10EDB80052524F525F4D4F44554C455F4E4F545F32
:10EDC800494E495449414C495A4544004E52465FC0
:10EDD8004552524F525F4D555445585F494E49541C
:10EDE8005F4641494C4544004E52465F4552524F9A
:10EDF800525F4D555445585F4C4F434B5F46414910
:10EE08004C4544004E52465F4552524F525F4D5555
:10EE18005445585F554E4C4F434B5F4641494C450E
:10EE280044004E52465F4552524F525F4D5554452D
:10EE3800585F434F4E445F494E49545F4641494CE1
:10EE48004544004E52465F4552524F525F4D4F4423
:10EE5800554C455F414C52454144595F494E4954D0
:10EE680049414C495A4544004E52465F4552524F1B
:10EE7800525F53544F524147455F46554C4C004EE4
:10EE880052465F4552524F525F4150495F4E4F5470
:10EE98005F494D504C454D454E544544004E5246F1
:10EEA8005F4552524F525F464541545552455F4E59
:10EEB8004F545F454E41424C4544004E52465F45D3
:10EEC80052524F525F494F5F50454E44494E47009A
:10EED8004E52465F4552524F525F4452565F545706
:10EEE800495F4552525F4F56455252554E004E5259
:10EEF800465F4552524F525F4452565F5457495FDE
:10EF08004552525F414E41434B004E52465F455277
:10EF1800524F525F4452565F5457495F4552525FB1
:10EF2800444E41434B004E52465F4552524F525F4A
:10EF3800424C455F495053505F52585F504B545FA5
:10EF48005452554E4341544544004E52465F455233
:10EF5800524F525F424C455F495053505F434841BE
:10EF68004E4E454C5F414C52454144595F455849C6
:10EF7800535453004E52465F4552524F525F424CD3
:10EF8800455F495053505F4C494E4B5F444953438A
:10EF98004F4E4E4543544544004E52465F455252EB
:10EFA8004F525F424C455F495053505F5045455260
:10EFB8005F52454A4543544544000000982F8A4211
:10EFC80091443771CFFBC0B5A5DBB5E95BC25639B3
:10EFD800F111F159A4823F92D55E1CAB98AA07D8CB
:10EFE800015B8312BE853124C37D0C55745DBE72EE
:10EFF800FEB1DE80A706DC9B74F19BC1C1699BE46E
:10F008008647BEEFC69DC10FCCA10C246F2CE92DFD
:10F01800AA84744ADCA9B05CDA88F97652513E9821
:10F028006DC631A8C82703B0C77F59BFF30BE0C628
:10F038004791A7D55163CA0667292914850AB727B6
:10F0480038211B2EFC6D2C4D130D385354730A6553
:10F05800BB0A6A762EC9C281852C7292A1E8BFA22A
:10F068004B661AA8708B4BC2A3516CC719E892D192
:10F07800240699D685350EF470A06A1016C1A41915
:10F08800086C371E4C774827B5BCB034B30C1C3914
:10F098004AAAD84E4FCA9C5BF36F2E68EE828F74D3
:10F0A8006F63A5781478C8840802C78CFAFFBE90ED
:10F0B800EB6C50A4F7A3F9BEF27871C6480028009B
:10F0C800002040002DA0020049880200EB870200C2
:10F0D8003D8D0200AF8D0200CF8D02002587020012
:10F0E800E5860200C58C020000000000433A5C6E11
:10F0F8006F726469635F73656D695C6E5246355FF4
:10F1080053444B5F31352E332E305F3539616333CD
:10F1180034355C636F6D706F6E656E74735C626FAF
:10F12800617264735C626F617264732E63001112A2
:10F13800102E2E2F2E2E2F2E2E2F2E2E2F2E2E2F00
:10F148006D6F64756C65732F6E7266782F68616C6D
:10F158002F6E72665F6770696F2E6800433A5C6E47
:10F168006F726469635F73656D695C6E5246355F83
:10F1780053444B5F31352E332E305F35396163335D
:10F1880034355C636F6D706F6E656E74735C6C693B
:10F19800627261726965735C63727970746F5C6EB8
:10F1A80072665F63727970746F5F736861726564A9
:10F1B8002E6300008922237E08D8BB1F65D20F2446
:10F1C800538AD762380829BF49C33B134C697F4F1C
:10F1D8004AE77589B9B534A62C96AD29CC75DFD721
:10F1E80087916DB21173553D57FEA3E22582B75B37
:10F1F800CA6BB8E452656365697665642061206608
:10F2080061756C74212069643A203078253038782B
:10F218002C2070633A203078253038782C20696E9D
:10F22800666F3A2030782530387800526563656912
:10F2380076656420616E206572726F723A2030784C
:10F2480025303878210000000338FDD87047496E12
:10F2580073696465206D61696E004166746572202A
:10F268006D61696E0000000008200001FFFFFFFFCC
:10F27800FFFFFFFFFFFFFFFF00000000000000008E
:10F288000000000001000000FFFFFFFF512563FCA4
:10F29800C2CAB9F3849E17A7ADFAE6BCFFFFFFFF09
:10F2A800FFFFFFFF00000000FFFFFFFF96C298D896
:10F2B8004539A1F4A033EB2D817D0377F240A46397
:10F2C800E5E6BCF847422CE1F2D1176BF551BF37A0
:10F2D8006840B6CBCE5E316B5733CE2B169E0F7C73
:10F2E8004AEBE78E9B7F1AFEE242E34F4B60D22740
:10F2F8003E3CCE3BF6B053CCB0061D65BC86987636
:10F3080055BDEBB3E7933AAAD835C65AF799020028
:10F318004D9B0200A99B02005465726D696E616C79
:10F32800005254540053454747455200526573658F
:10F338007474696E6720626F6F746C6F6164657254
:10F348002E000000000000000338FDD87047496E09
:10F3580061637469766974792074696D656F757411
:10F368002E00496E206E72665F626F6F746C6F61FB
:10F378006465725F696E697400426F6F74207661AC
:10F388006C69646174696F6E206661696C65642E6E
:10F39800204E6F2076616C69642061707020746FF4
:10F3A80020626F6F742E00426F6F742076616C69F3
:10F3B800646174696F6E206661696C65642E2053A0
:10F3C8006F66744465766963652069732070726539
:10F3D80073656E742062757420696E76616C6964F9
:10F3E8002E00426F6F742076616C69646174696F76
:10F3F8006E206661696C65642E20417070206973A7
:10F4080020696E76616C69642E00417070206973A2
:10F418002076616C696400444655206D6F646520F0
:10F428006265636175736520617070206973206E11
:10F438006F742076616C69642E00444655206D6FA8
:10F448006465207265717565737465642076696199
:10F458002047505245475245542E00444655206D8A
:10F468006F6465207265717565737465642076696B
:10F478006120626F6F746C6F61646572207365746C
:10F4880074696E67732E00556E7265616368616298
:10F498006C6500456E746572206D61696E206C6FD5
:10F4A8006F7000433A5C6E6F726469635F73656D79
:10F4B800695C6E5246355F53444B5F31352E332EAF
:10F4C800305F353961633334355C636F6D706F6EEF
:10F4D800656E74735C6C69627261726965735C6293
:10F4E8006F6F746C6F616465725C6E72665F626F79
:10F4F8006F746C6F616465722E6300696E20776546
:10F50800616B206E72665F6466755F696E69745FB1
:10F51800757365720052756E6E696E67206E7266DD
:10F528005F626F6F746C6F616465725F6170705F4A
:10F538007374617274207769746820616464726599
:10F5480073733A20307825303878004469736162E3
:10F558006C696E6720696E74657272757074732E4B
:10F56800204E5649432D3E494345525B305D3A2073
:10F5780030782578004661696C65642072756E6E16
:10F58800696E67206E72665F6466755F6D62725F32
:10F598006972715F666F72776172645F61646472C9
:10F5A8006573735F736574282900436F756C6420F5
:10F5B8006E6F742070726F7465637420626F6F74FD
:10F5C8006C6F6164657220616E6420736574746920
:10F5D8006E67732070616765732C20307825782EEC
:10F5E80000436F756C64206E6F742070726F746561
:10F5F800637420536F667444657669636520616E31
:10F6080064206170706C69636174696F6E2C20305E
:10F618007825782E0074696D65725F73746F702039
:10F628002830782578290074696D65725F6669727B
:10F6380065202830782578290000000000000000A7
:10F6480000000000000000000338FDD8704774690E
:10F658006D65725F616374697661746520283078BE
:10F6680025782900433A5C6E6F726469635F73653D
:10F678006D695C6E5246355F53444B5F31352E33AE
:10F688002E305F353961633334355C636F6D706F6D
:10F698006E656E74735C6C69627261726965735CC5
:10F6A800626F6F746C6F616465725C6E72665F62C4
:10F6B8006F6F746C6F616465725F6466755F74699F
:10F6C8006D6572732E6300566572696679696E6737
:10F6D80020424C3A20416464723A20307825303810
:10F6E800782C205372633A203078253038782C20D3
:10F6F8004C656E3A2030782530387800436F707941
:10F70800696E6720626F6F746C6F616465723A200E
:10F718005372633A203078253038782C204C656E47
:10F728003A20307825303878004E6F20626F6F7439
:10F738006C6F6164657220636F7079206E656564B3
:10F7480065642C20626F6F746C6F616465722075DC
:10F75800706461746520636F6D706C6574652E00EC
:10F768005265717565737420746F20636F707920AA
:10F77800424C206661696C6564004E6F20636F704F
:10F7880079206E656564656400433A5C6E6F7264E7
:10F7980069635F73656D695C6E5246355F53444BB0
:10F7A8005F31352E332E305F353961633334355C44
:10F7B800636F6D706F6E656E74735C6C6962726195
:10F7C800726965735C626F6F746C6F616465725C9B
:10F7D8006E72665F626F6F746C6F616465725F668C
:10F7E800775F61637469766174696F6E2E63004335
:10F7F8006F7079696E67203078257820746F2030B3
:10F808007825782C2073697A653A20307825780035
:10F818004661696C656420746F207772697465202D
:10F82800696D61676520636F7079696E67207072B2
:10F838006F677265737320746F2073657474696E73
:10F84800677320706167652E00456E746572206E5F
:10F8580072665F626F6F746C6F616465725F667702
:10F868005F61637469766174650056616C696420D0
:10F8780041707000456E746572206E72665F6466D2
:10F88800755F6170705F636F6E74696E7565005344
:10F89800657474696E672061707020617320766189
:10F8A8006C69640043524320636F6D7075746174B2
:10F8B800696F6E206661696C656420666F7220638B
:10F8C8006F70696564206170703A20737263206399
:10F8D80072633A203078253038782C20726573208E
:10F8E8006372633A203078253038780056616C6945
:10F8F800642053440056616C696420424C00566190
:10F908006C6964205344202B20424C00456E74657A
:10F9180072206E72665F6466755F73645F626C5FA7
:10F92800636F6E74696E75650053442B424C3A20C0
:10F93800534420636F7079206661696C6564005375
:10F94800442B424C3A20424C20636F707920666108
:10F95800696C6564004E6F206669726D77617265C7
:10F9680020746F2061637469766174652E00416349
:10F978007469766174696F6E206661696C6564206C
:10F9880077697468206572726F7220256420286216
:10F99800616E6B20636F64653A20307825782900A2
:10F9A8004120536F667444657669636520686173A6
:10F9B800206A757374206265656E20616374697668
:10F9C800617465642E2049742773206C696B656CBB
:10F9D80079207468617420616E206170706C69634D
:10F9E8006174696F6E2077696C6C20636F6D652038
:10F9F800696D6D6564696174656C7900436F756CD8
:10FA080064206E6F742077726974652073657474EE
:10FA1800696E67732E00456E746572206E72665F3C
:10FA2800626F6F746C6F616465725F6466755F7333
:10FA3800645F636F6E74696E756500536F7572638A
:10FA480065206164647265737320646F6573206EEA
:10FA58006F7420636F6E7461696E20612076616CCB
:10FA6800696420536F66744465766963652E005334
:10FA78004420616C726561647920636F70696564A4
:10FA8800005570646174696E672053442E204F6C72
:10FA980064205344207665723A2025642C204E65F4
:10FAA80077207665723A202564004661696C656442
:10FAB80020746F20636F7079206669726D77617248
:10FAC800652E0057445420656E61626C656420435E
:10FAD80052563A2564207469636B730053746172DB
:10FAE80074696E6720612074696D657220282564C9
:10FAF800207469636B732920666F7220666565647C
:10FB0800696E67207761746368646F672E00574475
:10FB180054206973206E6F7420656E61626C656431
:10FB2800006E72665F626F6F746C6F616465725F9E
:10FB380077647400496E7465726E616C20666565E1
:10FB480064000000EFB40200E9B40200C9B4020086
:10FB58002000000078000000000000000100010003
:10FB68000000000001000000000000000200050085
:10FB7800010000004200000000000000000000003A
:10FB8800000000000000000000000000010011005B
:10FB98000100FFFF01000000000000000200170044
:10FBA8000200FEFF64010000F4FB020000000000F8
:10FBB800000000000000000000000000010001003B
:10FBC8000000000001000000000000000200050025
:10FBD80001000000220000000000000000000000FA
:10FBE80000000000000000000000000001001100FB
:10FBF8000400FCFF040000000000000002001100E7
:10FC08000400FCFF040000000000000003002100C5
:10FC18000400FCFF040010000000000004001100B4
:10FC28000100FFFF010000000000000005001100B6
:10FC38000200FEFF040000000000000006001100A2
:10FC48000400FCFF04000000000000000700110091
:10FC58000400FCFF0400000000000000080017007A
:10FC68000200FEFF24000000C4FB0200090010008F
:10FC78000100FFFF01000000A4FC02000A002700A9
:10FC88000200FEFF4400030064FB020000000000C5
:10FC9800000000000000000000000000000000005C
:10FCA800010017000400FCFF6801000094FB02003B
:10FCB800020017000400FCFFAC010000D8FC0200A1
:10FCC800000000000000000000000000000000002C
:10FCD80001000700000000006801000094FB02001A
:10FCE8000200010000000000010000000000000008
:10FCF80003000500010000004200000000000000B1
:10FD080000000000000000000000000000000000EB
:10FD1800456E746572696E6720444655206D6F6440
:10FD2800652E00436F756C64206E6F7420696E6970
:10FD380074616C697A6520444655207472616E73EB
:10FD4800706F72743A203078253038780050EADACB
:10FD5800308883B89F604F15F30000C98E416476E0
:10FD68006572746973696E672E2E2E00433A5C6E55
:10FD78006F726469635F73656D695C6E5246355F67
:10FD880053444B5F31352E332E305F353961633341
:10FD980034355C636F6D706F6E656E74735C6C691F
:10FDA800627261726965735C626F6F746C6F6164B3
:10FDB80065725C626C655F6466755C6E72665F64D2
:10FDC80066755F626C652E630044465520726571E6
:10FDD80075657374202564206661696C6564207795
:10FDE800697468206572726F723A203078257800DD
:10FDF8005368757474696E6720646F776E20424C1F
:10FE080045207472616E73706F72742E004469734A
:10FE1800636F6E6E656374696E672E00424C452091
:10FE28007472616E73706F72742073687574206475
:10FE38006F776E2E004466755461726700496E696B
:10FE48007469616C697A696E6720424C4520444642
:10FE580055207472616E73706F7274005365747498
:10FE6800696E6720757020766563746F722074619F
:10FE7800626C653A2030782530387800456E6162CA
:10FE88006C696E6720536F66744465766963652E86
:10FE980000436F6E6669677572696E6720424C45EC
:10FEA80020737461636B2E00456E61626C696E67C6
:10FEB8002074686520424C4520737461636B2E0082
:10FEC8004E6F206164766572746973696E67206E1F
:10FED800616D6520666F756E640053657474696E34
:10FEE8006720616476206E616D653A2025732C2049
:10FEF8006C656E6774683A202564005573696E678F
:10FF08002064656661756C742061647665727469D5
:10FF180073696E67206E616D6500424C45204446EA
:10FF280055207472616E73706F727420696E697493
:10FF380069616C697A65642E00436F6E6E656374DF
:10FF48006564004661696C75726520746F20757010
:10FF58006461746520636F6E6E656374696F6E208B
:10FF6800706172616D65746572733A2030782578B6
:10FF78000063616E6E6F7420616C6C6F6361746591
:10FF8800206D656D6F7279206275666665722100F5
:10FF980042756666657220257020616371756972A5
:10FFA80065642C206C656E20256420282564290052
:10FFB800526563656976656420424C455F474154E4
:10FFC80054535F4556545F45584348414E47455F33
:10FFD8004D54555F5245515545535420287265710B
:10FFE800756573743A2025642C207265706C793AB3
:08FFF800202564292E0052654A
:020000023000CC
:1000000063656976656420424C455F4741505F45B2
:1000100056545F444154415F4C454E4754485F55E8
:1000200050444154455F524551554553542E00525A
:100030006563656976656420424C455F4741505F62
:100040004556545F444154415F4C454E4754485FC8
:10005000555044415445202825752C206D61785F0A
:1000600072785F74696D65202575292E005265636D
:10007000656976656420424C455F4741505F45564F
:10008000545F5345435F504152414D535F52455178
:1000900055455354004343434420666F72207365B3
:1000A0007276696365206368616E67656420697351
:1000B0002030782530347800526563656976656450
:1000C00020424C455F4741505F4556545F434F4E79
:1000D0004E5F504152414D5F555044415445006D73
:1000E00061785F636F6E6E5F696E74657276616C66
:1000F0003A202564006D696E5F636F6E6E5F696E96
:1001000074657276616C3A20256400736C61766563
:100110005F6C6174656E63793A20256400636F6E6D
:100120006E5F7375705F74696D656F75743A2025C5
:100130006400526563656976656420424C455F479B
:1001400041505F4556545F434F4E4E5F50415241C0
:100150004D5F5550444154455F52455155455354A8
:10016000004661696C75726520746F2075706461FA
:10017000746520636F6E6E656374696F6E20706165
:1001800072616D6574657220726571756573743A1C
:100190002030782578005265636569766564204271
:1001A0004C455F4741505F4556545F5048595F5535
:1001B0005044415445202852583A25642C20545824
:1001C0003A25642C207374617475733A2564290090
:1001D000526563656976656420424C455F474150CE
:1001E0005F4556545F5048595F5550444154455FF0
:1001F000524551554553542E005365742072656322
:1002000065697074206E6F74696600436F756C6405
:10021000206E6F742068616E646C65206F6E5F6322
:1002200074726C5F70745F77726974652E2065728A
:10023000725F636F64653A203078253034780052FD
:100240006563656976656420424C455F4741505F50
:100250004556545F5345435F494E464F5F524551A3
:10026000554553540046696E69736865642068613A
:100270006E646C696E6720636F6E6E2073656320B9
:1002800075706461746500000000000000000000EB
:100290000338FDD870470C000C000000580246726D
:1002A0006565696E672062756666657220257000F7
:1002B0006E72665F6466755F626C65007772697402
:1002C0006500657261736500466C61736820257313
:1002D00020737563636573733A20616464723D25AE
:1002E000702C2070656E64696E6720256400466C12
:1002F000617368202573206661696C65642028300D
:10030000782578293A20616464723D25702C206C30
:10031000656E3D307825782062797465732C207085
:10032000656E64696E67202564006E72665F667331
:10033000746F726167655F6572617365286164647B
:10034000723D307825702C206C656E3D25642070E0
:1003500061676573292C20717565756520757361FA
:1003600067653A202564006E72665F6673746F720B
:100370006167655F65726173652829206661696CD4
:1003800065642077697468206572726F72203078B6
:1003900025782E00496E697469616C697A696E67A7
:1003A000206E72665F6673746F726167655F7364F7
:1003B000206261636B656E642E00496E69746961C9
:1003C0006C697A696E67206E72665F6673746F72AD
:1003D0006167655F6E766D63206261636B656E64F5
:1003E0002E006E72665F6673746F726167655F7709
:1003F0007269746528616464723D25702C20737283
:10040000633D25702C206C656E3D256420627974F7
:100410006573292C20717565756520757361676535
:100420003A202564006E72665F6673746F7261674E
:10043000655F77726974652829206661696C6564F7
:100440002077697468206572726F72203078257821
:100450002E006E72665F6466755F666C617368001D
:100460005363686564756C65722072616E206F7588
:1004700074206F662073706163652100433A5C6E7F
:100480006F726469635F73656D695C6E5246355F58
:1004900053444B5F31352E332E305F353961633332
:1004A00034355C636F6D706F6E656E74735C6C6910
:1004B000627261726965735C626F6F746C6F6164A4
:1004C00065725C6466755C6E72665F6466755F72A9
:1004D00065715F68616E646C65722E630048616E61
:1004E000646C65204E52465F4446555F4F505F52E4
:1004F0004543454950545F4E4F5449465F53455418
:100500000048616E646C65204E52465F4446555FFC
:100510004F505F41424F52540048616E646C6520F9
:100520004E52465F4446555F4F505F4F424A4543E7
:10053000545F4352454154452028636F6D6D616E91
:1005400064290048616E646C65204E52465F4446E3
:10055000555F4F505F4352435F4745542028636FB8
:100560006D6D616E64290048616E646C65204E5249
:10057000465F4446555F4F505F4F424A4543545F84
:1005800057524954452028636F6D6D616E64290090
:1005900048616E646C65204E52465F4446555F4F1D
:1005A000505F4F424A4543545F4558454355544573
:1005B0002028636F6D6D616E6429005772697469DC
:1005C0006E672076616C696420696E697420636F60
:1005D0006D6D616E6420746F20666C6173682E00AF
:1005E00048616E646C65204E52465F4446555F4FCD
:1005F000505F4F424A4543545F53454C4543542056
:1006000028636F6D6D616E64290048616E646C656E
:10061000204E52465F4446555F4F505F4F424A4519
:1006200043545F4352454154452028646174612915
:100630000043616E6E6F742063726561746520643F
:10064000617461206F626A65637420776974686F92
:1006500075742076616C696420696E697420636FBB
:100660006D6D616E64004F626A6563742073697AB0
:10067000652063616E6E6F7420626520302E004FBE
:10068000626A6563742073697A65206D757374207E
:100690006265207061676520616C69676E656400E2
:1006A000496E76616C69642073697A6520666F7241
:1006B000206F626A6563742028746F6F206C6172AA
:1006C000676529004372656174696E6720746865A7
:1006D000206F626A65637420776974682073697A31
:1006E000652030782530387820776F756C64206FFE
:1006F000766572666C6F77206669726D7761726578
:100700002073697A652E204F66667365742069735D
:100710002030782530387820616E64206669726DEB
:10072000776172652073697A652069732030782556
:100730003038782E004572617365206F7065726184
:1007400074696F6E206661696C65640043726561EF
:1007500074696E67206F626A656374207769746874
:100760002073697A653A2025642E204F666673658A
:10077000743A203078253038782C204352433A2080
:100780003078253038780048616E646C65204E52B0
:10079000465F4446555F4F505F4F424A4543545F62
:1007A0005752495445202864617461290057726981
:1007B0007465207265717565737420746F6F206C39
:1007C0006F6E670048616E646C65204E52465F44F0
:1007D00046555F4F505F4352435F4745542028645E
:1007E00061746129004F66667365743A25642C2034
:1007F0004352433A3078253038780048616E646C53
:1008000065204E52465F4446555F4F505F4F424A07
:100810004543545F45584543555445202864617409
:10082000612900496E76616C696420646174612E8F
:100830002065787065637465643A2025642C2067B0
:100840006F743A2025640048616E646C65204E52D6
:10085000465F4446555F4F505F4F424A4543545FA1
:1008600053454C45435420286461746129006372E8
:1008700063203D20307825782C206F666673657480
:10088000203D20307825782C206D61785F73697A5F
:1008900065203D203078257800496E76616C69646A
:1008A000206F626A656374207479706520696E20B8
:1008B000726571756573742E00496E76616C69643A
:1008C000206F70636F646520726563656976656427
:1008D0003A20307825782E004661696C6564207472
:1008E0006F207363686564756C65206F626A656309
:1008F0007420657865637574653A20307825782EA4
:100900000057686F6C65206669726D77617265204B
:10091000696D6167652072656365697665642E201F
:10092000506F737476616C69646174696E672E00D0
:10093000526571756573742068616E646C696E6769
:1009400020636F6D706C6574652E20526573756CD5
:10095000743A203078257800416C6C20666C6173A5
:1009600068206F7065726174696F6E73206861765C
:100970006520636F6D706C657465642E2044465508
:1009800020636F6D706C657465642E006E72665FB7
:100990006466755F7265715F68616E646C65720034
:1009A00043616C6C696E67206E72665F6466755F2A
:1009B00073657474696E67735F696E697428292E34
:1009C0002E2E006E72665F6466755F666C6173687A
:1009D0005F696E69742829206661696C6564207797
:1009E000697468206572726F723A202578005573B9
:1009F000696E672073657474696E677320706167D0
:100A0000652E00436F7079696E6720666F72626948
:100A10006464656E2070617274732066726F6D20FD
:100A20006261636B757020706167652E005265733B
:100A3000746F72696E672073657474696E67732072
:100A400066726F6D206261636B75702073696E638F
:100A500065207468652073657474696E67732070AF
:100A600061676520636F6E74656E74732061726573
:100A700020696E76616C6964202843524320657258
:100A8000726F72292E00526573657474696E6720E7
:100A9000626F6F746C6F61646572207365747469E2
:100AA0006E67732073696E6365206E65697468652F
:100AB00072207468652073657474696E6773207042
:100AC000616765206E6F7220746865206261636B78
:100AD0007570206172652076616C696420284352CC
:100AE00043206572726F72292E004F6C642073650B
:100AF0007474696E677320706167652064657465DE
:100B0000637465642E20557067726164696E672036
:100B1000696E666F2E006E72665F6466755F7365E0
:100B20007474696E67735F77726974655F616E6410
:100B30005F6261636B75702829206661696C65640A
:100B40002077697468206572726F723A2025780088
:100B50004261636B696E6720757020736574746998
:100B60006E6773207061676520746F2061646472C2
:100B700065737320307825782E00433A5C6E6F726F
:100B80006469635F73656D695C6E5246355F53449B
:100B90004B5F31352E332E305F3539616333343559
:100BA0005C636F6D706F6E656E74735C6C6962729E
:100BB00061726965735C626F6F746C6F616465729A
:100BC0005C6466755C6E72665F6466755F7365749F
:100BD00074696E67732E6300436F756C64206E6F6B
:100BE0007420706572666F726D206261636B7570E0
:100BF000206F6620626F6F746C6F61646572207322
:100C0000657474696E677321204572726F723A2041
:100C1000307825780044657374696E6174696F6E0D
:100C20002073657474696E677320617265206964EE
:100C3000656E746963616C20746F20736F75726385
:100C4000652C207772697465206E6F74206E6565FF
:100C50006465642E20536B697070696E672E00574F
:100C6000726974696E672073657474696E67732E38
:100C70002E2E0045726173696E67206F6C6420735D
:100C8000657474696E67732061743A20307825301A
:100C9000387800436F756C64206E6F7420657261E4
:100CA0007365207468652073657474696E6773205A
:100CB000706167652100436F756C64206E6F7420EE
:100CC00077726974652074686520444655207365A1
:100CD0007474696E6773207061676521006E726657
:100CE0005F6466755F73657474696E6773004572DF
:100CF0006173696E672073657474696E67732070C1
:100D0000616765206164646974696F6E616C2064F9
:100D10006174612E006E72665F6466755F736574E0
:100D200074696E67735F7376636900536875747472
:100D3000696E6720646F776E207472616E73706F76
:100D40007274732028666F756E643A2025642900DA
:100D50004661696C656420746F2073687574646F94
:100D6000776E207472616E73706F72742025642CBC
:100D7000206572726F7220256400496E6974696122
:100D80006C697A696E67207472616E73706F7274C9
:100D9000732028666F756E643A20256429004661C9
:100DA000696C656420746F20696E697469616C692F
:100DB0007A65207472616E73706F72742025642C72
:100DC000206572726F7220256400456E7465722012
:100DD0006E72665F6466755F63616368655F70729B
:100DE0006570617265282900726571756972656444
:100DF0005F73697A653A20307825782E00747275B1
:100E0000650066616C73650073696E676C655F622F
:100E1000616E6B3A2025732E006B6565705F6170A3
:100E2000703A2025732E006B6565705F736F667472
:100E30006465766963653A2025732E0053445F50DC
:100E4000524553454E543A2025732E0042616E6B35
:100E500020636F6E74656E74733A0042616E6B202E
:100E60003020636F64653A203078253032783A203C
:100E700053697A653A20307825780042616E6B209C
:100E80003120636F64653A203078253032783A201B
:100E900053697A653A203078257800433A5C6E6F62
:100EA000726469635F73656D695C6E5246355F534A
:100EB000444B5F31352E332E305F35396163333427
:100EC000355C636F6D706F6E656E74735C6C6962B8
:100ED0007261726965735C626F6F746C6F61646577
:100EE000725C6466755C6E72665F6466755F75746D
:100EF000696C732E6300706173733A2025642E0051
:100F000063616368655F616464726573733A20301E
:100F10007825782E0063616368655F746F6F5F7317
:100F20006D616C6C3A2025732E006B6565705F6691
:100F300069726D776172653A2025732E0064656C65
:100F40006574655F6D6F72653A2025732E0041628E
:100F50006F7274696E672E2043616E6E6F742066C7
:100F60006974206E6577206669726D77617265209D
:100F70006F6E2064657669636500496E76616C69A1
:100F8000646174696E67206170702E006E72665FB6
:100F900063727970746F5F686173685F63616C63BB
:100FA000756C6174652829206661696C65642077B9
:100FB000697468206572726F7220257300496E76BD
:100FC000616C696420626F6F742076616C69646122
:100FD00074696F6E20747970653A20256400433A15
:100FE0005C6E6F726469635F73656D695C6E5246B7
:100FF000355F53444B5F31352E332E305F353961C9
:10100000633334355C636F6D706F6E656E74735CE3
:101010006C69627261726965735C626F6F746C6F28
:10102000616465725C6466755C6E72665F64667549
:101030005F76616C69646174696F6E2E63006D61C7
:101040006A6F72006D696E6F7200536F66744465EB
:1010500076696365207570646174652069732061C9
:101060002025732076657273696F6E2075706461D8
:1010700074652E2043757272656E743A2025642E55
:10108000204E65773A2025642E0043524320636842
:1010900065636B206F6620617070206661696C65A6
:1010A000642E2052657475726E2025640048617349
:1010B0006820766572696669636174696F6E2E2057
:1010C000737461727420616464726573733A203062
:1010D0007825782C2073697A653A20307825780055
:1010E000436F756C64206E6F742072756E2068613A
:1010F000736820766572696669636174696F6E20D2
:10110000286572725F636F64652030782578292EB8
:101110000048617368207665726966696361746905
:101120006F6E206661696C65642E0045787065633A
:1011300074656420465720686173683A004163749F
:1011400075616C20465720686173683A00496E6982
:101150007420636F6D6D616E64206C61726765727F
:10116000207468616E2065787065637465642E0014
:101170004578656375746520776974682066617564
:101180006C7479206F66667365740043616E2774B2
:101190002066696E6420726F6F6D20666F722075B5
:1011A000706461746500577269746520616464726B
:1011B0006573732073657420746F20307825303820
:1011C00078004661696C656420746F206465636FA4
:1011D000646520696E6974207061636B657400508A
:1011E000726576616C69646174696F6E20666169AD
:1011F0006C65642E00496E697420636F6D6D616E5D
:10120000643A005369676E61747572652072657126
:1012100075697265642E20436865636B696E67202B
:101220007369676E61747572652E004E6F20736905
:10123000676E617475726520666F756E642E004905
:101240006E76616C6964207369676E61747572652E
:1012500020747970650043616C63756C6174696EAC
:1012600067206861736820286C656E3A20256429C0
:1012700000566572696679207369676E617475726C
:1012800065005369676E6174757265206661696C8B
:10129000656420286572725F636F64653A203078F8
:1012A000257829005369676E61747572653A004844
:1012B0006173683A005075626C6963204B65793AD6
:1012C00000496D61676520766572696669656400CD
:1012D00050423A20496E6974207061636B657420D6
:1012E00064617461206C656E3A20256400496E76F5
:1012F000616C69646174696E67206F6C64206170F1
:10130000706C69636174696F6E20696E2062616ED2
:101310006B20302E0054686520536F6674446576E8
:1013200069636520646F6573206E6F7420636F6EF0
:101330007461696E20746865206D61676963206EF1
:10134000756D626572206964656E74696679696E2F
:1013500067206974206173206120536F667444654F
:10136000766963652E0054686520536F6674446522
:10137000766963652073697A6520696E2074686593
:1013800020696E666F2073747275637420697320B0
:10139000746F6F20736D616C6C20636F6D70617220
:1013A00065642077697468207468652073697A655C
:1013B000207265706F7274656420696E2074686550
:1013C00020696E697420636F6D6D616E642E0049D3
:1013D0006E76616C69646174696E672061707020FB
:1013E0006265636175736520697420697320696E35
:1013F000636F6D70617469626C65207769746820D1
:1014000074686520536F66744465766963652E0061
:101410004D616A6F72205344207570646174652059
:10142000627574206E6F20424C2E2041626F727480
:1014300020746F2061766F696420696E63617061EA
:101440006369746174696E672074686520424C2E0C
:1014500000426F6F742076616C69646174696F6EAD
:10146000206F6620626F6F746C6F616465722069B3
:1014700073206E6F7420737570706F727465642062
:10148000616E642077696C6C2062652069676E6F9D
:101490007265642E0048616E646C65723A20496E14
:1014A00076616C69642070726F746F636F6C206218
:1014B0007566666572206D5F70625F7374726561D8
:1014C0006D0048616E646C65723A20496E76616C9D
:1014D000696420696E697420636F6D6D616E642E3E
:1014E0000048616E646C65723A20496E76616C6981
:1014F000642070726F746F636F6C206275666665CE
:1015000072206D5F70625F73747265616D2028690F
:101510006E697420636F6D6D616E6429006E726612
:101520005F6466755F76616C69646174696F6E0093
:10153000424C2073697A652028256429206F7665DE
:1015400072206C696D6974202825642900496E69D0
:1015500074207061636B657420646F6573206E6FB7
:101560007420636F6E7461696E2076616C696420AB
:101570006669726D776172652073697A6500433AB6
:101580005C6E6F726469635F73656D695C6E524611
:10159000355F53444B5F31352E332E305F35396123
:1015A000633334355C636F6D706F6E656E74735C3E
:1015B0006C69627261726965735C626F6F746C6F83
:1015C000616465725C6466755C6E72665F646675A4
:1015D0005F7665725F76616C69646174696F6E2EA7
:1015E0006300496E76616C6964206669726D77612B
:1015F000726520747970652E00496E76616C69643D
:10160000206861736820747970652E004E6F2048E1
:10161000572076657273696F6E2E004661756C7423
:10162000792048572076657273696F6E2E00534497
:1016300020726571206E6F74206D65742E004657A0
:101640002076657273696F6E20746F6F206C6F7790
:101650002E0046572076657273696F6E206D697330
:1016600073696E672E006E72665F6466755F76657D
:10167000725F76616C69646174696F6E000100006D
:1016800007000000FCE5020004E60200080000007C
:101690000CE602001CE602000800000004E602005E
:1016A0000CE60200080000006E72665F736468005A
:1016B00073645F626C655F6366675F736574282936
:1016C0002072657475726E65642025732077686575
:1016D0006E20617474656D7074696E6720746F201C
:1016E00073657420424C455F434F4E4E5F434647FF
:1016F0005F4741502E0073645F626C655F6366678D
:101700005F73657428292072657475726E65642034
:101710002573207768656E20617474656D707469D7
:101720006E6720746F2073657420424C455F47419B
:10173000505F4346475F524F4C455F434F554E54B1
:101740002E0073645F626C655F6366675F736574C8
:1017500028292072657475726E6564202573207760
:1017600068656E20617474656D7074696E6720744D
:101770006F2073657420424C455F434F4E4E5F436C
:1017800046475F474154542E0073645F626C655F47
:101790006366675F73657428292072657475726E5D
:1017A0006564202573207768656E20617474656DAB
:1017B0007074696E6720746F2073657420424C45A5
:1017C0005F434F4D4D4F4E5F4346475F56535F5506
:1017D0005549442E0073645F626C655F6366675FA2
:1017E00073657428292072657475726E656420258E
:1017F00073207768656E20617474656D7074696EAE
:101800006720746F2073657420424C455F474154D4
:1018100054535F4346475F415454525F5441425FC3
:1018200053495A452E0073645F626C655F63666757
:101830005F73657428292072657475726E65642003
:101840002573207768656E20617474656D707469A6
:101850006E6720746F2073657420424C455F47416A
:101860005454535F4346475F534552564943455F7F
:101870004348414E4745442E00496E73756666697C
:101880006369656E742052414D20616C6C6F6361B9
:1018900074656420666F722074686520536F667487
:1018A0004465766963652E004368616E67652074E0
:1018B00068652052414D207374617274206C6F63AF
:1018C0006174696F6E2066726F6D203078257820A4
:1018D000746F20307825782E004D6178696D756DB4
:1018E0002052414D2073697A6520666F72206170C5
:1018F000706C69636174696F6E206973203078253C
:10190000782E0073645F626C655F656E61626C6502
:1019100028292072657475726E65642025732E0007
:10192000F4E50200FCE50200080000006E72665F4C
:101930007364685F626C65001CE6020024E60200C6
:10194000080000006E72665F7364685F736F630007
:10195000202020202020202020682828282820201F
:101960002020202020202020202020202020202077
:10197000481010101010101010101010101010102F
:1019800084848484848484848484101010101010CF
:101990001081818181818101010101010101010128
:1019A00001010101010101010101011010101010DC
:1019B00010828282828282020202020202020202F9
:1019C00002020202020202020202021010101020A1
:1019D0000007032004170201085710408000000090
:1019E000841B0300481A03005C1B030053756E0040
:1019F0004D6F6E005475650057656400546875003E
:101A00004672690053617400000000004A616E0074
:101A1000466562004D617200417072004D6179004F
:101A20004A756E004A756C00417567005365700019
:101A30004F6374004E6F7600446563000000000041
:101A4000414D00504D000000801B03007C1B030033
:101A50007C1B03007C1B03007C1B03007C1B03001E
:101A60007C1B03007C1B03007C1B03007C1B03000E
:101A7000FFFFFFFFFFFFFFFFFFFFFFFFFFFF000074
:101A8000BC1A0300EC190300F81A03000C1A030037
:101A9000401A0300A01A0300501B0300AC1A0300F5
:101AA000256D2F25642F2579000000002561202554
:101AB00062202565202554202559000053756E6449
:101AC0006179004D6F6E646179005475657364616E
:101AD00079005765646E6573646179005468757246
:101AE0007364617900467269646179005361747549
:101AF00072646179000000004A616E75617279005C
:101B00004665627275617279004D61726368004169
:101B10007072696C004D6179004A756E65004A7596
:101B20006C79004175677573740053657074656DE9
:101B3000626572004F63746F626572004E6F766506
:101B40006D62657200446563656D626572000000D8
:101B500025483A254D3A255300000000B5E2020021
:101B6000D1E20200DDE20200E9E2020005E3020048
:101B700011E302001DE302002BE30200000000005D
:101B80002E00000043000000504F53495800000051
:101B900000000000FF000000000000000000000046
:101BA0000000000000000000000000000000000035
:101BB0000000000001000000D4570020E45700207E
:101BC0000090D003FF00FFFF0100000000E00700CD
:101BD000E0190300E0190300E0190300E019030015
:041BE000E019030005
:0400000320006379FD
:00000001FF
